:020000040000FA
:0400000011EF04F008
:0800080054EF04F0156A196AB7
:10001000186E010E02D0186E040E0E6E1950155C8B
:1000200002E11850145C040ED8B0010ED8B4020ED0
:100030000E14D8A4010E12000B6A1C6E1D6A0096E5
:100040000B50D8B40086040E0A6E1D3805D81D501A
:1000500003D81C3801D81C500F0BF60FD8B0070F6F
:100060000A0F21D00B6A1C6E1D6A00960B50D8B483
:100070000086050E0A6E270E196E100E0CD8030EA0
:10008000196EE80E08D8196A640E05D8196A0A0EA6
:1000900002D81C5008D0186E1D50156E1C50146EDE
:1000A000E3EC02F01450146E0A4E00960B5003E07D
:1000B0000A5CD8B007D01450D8A4009600B602D07D
:1000C000300F06D1120000960B5003E100860A0E95
:1000D0000B6E2AC017F029C016F028C015F027C0F3
:1000E00014F00A6A1F6A1E6A1D6A0A0E1C6EFCD989
:1000F0000A2A0A500B5CD8A4F5D71C50D8A4009645
:1001000000A602D00B2C03D01C50300FE1D80B2ED0
:10011000E0D71200A66AA68E0900F55002E002D8C8
:10012000FBD71200216E89980000899A9298929AC2
:10013000F00E9216215000B21ED03A0E156E980E97
:10014000C9D9330E206E2AD8130E156E880EC2D967
:1001500025D8640EBED922D8640EBBD9220E206EDB
:100160001DD8280E07D80C0E05D8060E03D800821D
:10017000215001D00080206E00A00AD0899A030887
:100180000BE30AD8070E156ED00EA4D9D880120042
:100190000080FE0811E0898A203A00A0009089883A
:1001A000F00E801620500F0B80128998203A00B074
:1001B000F5D7320E8ED9D8802150120008C014F025
:1001C00009C015F0010E186E196A0F0EEA6E05C00F
:1001D000E9FF00002AD8D8A015D0182EFAD7FF0EB4
:1001E0001926D8B0F6D71426D8A01526D8A0120004
:1001F000C80E186E196AEDD70F0EEA6E05C0E9FF3A
:1002000014D8FEE255D8226A080E196E52D80DD8BD
:10021000D8B0223E1832192EF9D724AA226A24BA5D
:10022000189E47D8D88018501200120EE9260C509C
:10023000EF1205C0E9FFEF1424BC0C18FF0F1200E9
:10024000206E0F0EEA6EE26E0550E96E120FE16E3F
:10025000800E0E16080E216ED890D8B00E3E11D822
:100260002032212EFAD7000024BA0E300AD800D04E
:1002700000D000D0D88005D80950196E08501DD97B
:10028000120024AE0BD0EF500C1024AC0C18EF6E03
:10029000E7500C10D8A00C18E76E0BD0EF500C10E4
:1002A000D8A00C1824BC0C18EF6E0C1CE71601D05B
:1002B0000E8C24501F0B000F156E23500D0FD8B05D
:1002C000152A0EAC07D10E9C146E020EF5D902D180
:1002D00001BE28D701BAB4D701A202D001B075D0AF
:1002E000080E0EB4010E196E186A0F0EEA6E05C0E4
:1002F000E9FF0C50E5D90C50EF12090EEAD80C506A
:1003000005C0E9FFEF14FF0F0EA418320EB4183623
:100310003C0EDFD8192EEDD71850D8801200186E79
:10032000080E0EB4010E196E0F0EEA6E05C0E9FF3D
:100330000C50C6D90C501832D8B0EF123C0EC9D8A8
:100340000C50EF12192EF2D7D88012000EA21DD039
:1003500003D00E6E0EA019D00F0EEA6E05C0E9FF95
:100360000C50AED9010E156EF40EB4D80C50EF122D
:10037000640EAFD805C0E9FFEF500C14D890D8A494
:100380001200010E156E900EA5D8D88012000088BC
:1003900000A8009800BA03D0008A35D829E200945A
:1003A000080E196E40D81836192EFCD700B407D0A5
:1003B00000B801D04AD845D841D800B819D843D898
:1003C000D89018501CD0008800A8009800BC05D018
:1003D000FE0B0E6E008CD89012D000BE05D0206EA1
:1003E000008E11D805E2205012D802E200A807D0F2
:1003F0002CD827D8009C009E009A009424D82280F4
:10040000D8A02290120017D80E5000BA0109186E19
:10041000080E196E183617D801E217D812D80ED860
:10042000192EF8D710D80DD800D00000D89082B877
:10043000D88004D8120007D804D807D8829694969A
:1004400006D0948604D0948802D08B989498120099
:100450001C6E0F0EEA6E0550120FE96E0C50EF1273
:1004600005C0E9FFEF1425A00C1810E01C6607D0AA
:100470002350FF0F0CE3320E1FD8235008D01C2846
:10048000FF0E04E01C2C02D0245001D0261E263280
:100490001200A96EA66AA680A850A92A1200A86E0A
:1004A000A66AA684550EA76EAA0EA76EA682A6B24D
:1004B000FED7A694A92A1200196A186EFF0E1826F4
:1004C000192200D0D8A01200030E156EE60E02D835
:1004D000F5D7156AFB0F146E00D0E86A01D0140638
:1004E000155AFDE20000120017501F18800BF46E21
:1004F00017AE06D0D880000E14561556165617564D
:100500001FAE06D0D880000E1C561D561E561F5614
:10051000186A196A1A6A1B6A2D6A2E6A2F6A306A6B
:100520001F501E101D101C1023E0200EF36ED890DB
:1005300014361536163617362D362E362F363036FB
:100540001C502D5C1D502E581E502F581F503058D7
:1005500009E31C502D5E1D502E5A1E502F5A1F505D
:10056000305AD880183619361A361B36F32EDFD794
:10057000F4AE06D0D880000E185619561A561B56DF
:1005800018C014F019C015F01AC016F01BC017F0EF
:100590002DC01CF02EC01DF02FC01EF030C01FF06B
:1005A0001200196A186E14C020F01CC014F020C08C
:1005B0001CF015C020F01DC015F020C01DF005D0A6
:1005C000156A196A186E1D6A1C6A100EF36E1534CE
:1005D0001C361D3618501C5C19501D5805E3185068
:1005E0001C5E19501D5AD88014361536F32EEFD7DD
:1005F0001450120017C030F016C02FF015C02EF0A6
:1006000014C02DF02F501C02F3CF16F0F4CF17F0CA
:100610002E501D02F3501626F45017222D501E02A4
:10062000F3501626F450172230501C02F3501726B0
:100630002F501D02F35017262E501E02F35017267E
:100640002D501F02F35017262D501C02F3CF14F02B
:10065000F4CF15F02E501C02F3501526F45016223C
:10066000000E17222D501D02F3501526F4501622AD
:10067000000E1722120018502002F4CF1DF0F3CF05
:100680001CF019502102F4CF15F0F3CF14F01850DC
:100690002102F3501D26F4501422E86A1522195045
:1006A0002002F3501D26F4501422E86A15221C5033
:1006B0001200D89015321432FF0FFBE214501200D2
:1006C000FF0AEF1600D0E988E92AEC161200742020
:1006D000696E742E000074206578742E0000204B23
:1006E0004C5A20200000204E554C4C200000204E3B
:1006F000554C4C2000007420696E742E000074204C
:100700006578742E00002020202020200000455213
:10071000522044454D4F0000436F6E6E6563740078
:10072000746F204D494B41530000436F6D6D756EE2
:1007300069630000202044454D4F20200000202008
:1007400044454D4F20200000202020202020202044
:100750000000204D2031302E3300204D31302E331B
:100760002B0020204D372E360000204D2031312E19
:100770003400202044454D4F2020000020204445D7
:100780004D4F20200000202044454D4F20200000E8
:10079000202044454D4F20200000202044454D4F4F
:1007A00020200000202044454D4F20200000202024
:1007B00044454D4F20200000202044454D4F20202F
:1007C0000000202044454D4F20200000436F6E6EF6
:1007D00065637400202044454D4F202000002020F8
:1007E00044454D4F20200000202044454D4F2020FF
:1007F0000000202044454D4F20200000202044458B
:100800004D4F202000004B6C7A2044454D4F000096
:10081000202044454D4F202000002076322E3237D4
:100820000000F86A006AAB6A00010F0EC16E929078
:100830009292929492969298929A93909392939481
:1008400093869388938A938C938EF16AC00EF26E8E
:10085000F06A9E6AA16A9D6A010EA06E9F6AA26AF2
:10086000CD8ECD8CCD8ACD88CD96CD94CD92BA6AE1
:10087000BA86BA94BA82BA80030EBC6EE80EBB6E1A
:10088000CD8094909482948494969488948A949C35
:10089000948E06EE00F0ED6AE950EA10FCE1EF6A92
:1008A00082808180819227D0D8CF32F0336EE0CF22
:1008B00002F0E9CF03F0EACF04F00001A1A011D0CB
:1008C0000101012BFA0E015D00010AE10101016B3A
:1008D000D8920001E6A9D882D8B2E689D8A2E699D2
:1008E000A19003C0E9FF04C0EAFF02C0E0FF33505B
:1008F00032C0D8FF1000590E49EC02F0E96F5A0ED1
:1009000049EC02F0EA6F5B0E49EC02F0EB6F5C0E13
:1009100049EC02F0EC6F5D0E49EC02F0ED6F5E0EFB
:1009200049EC02F0EE6F5F0E49EC02F0EF6F600EE3
:1009300049EC02F0F06F650E49EC02F03A6E660E7B
:1009400049EC02F03B6E4AEC02F03C6E4AEC02F0DD
:100950003D6E4AEC02F03E6E6A0E49EC02F0406ECB
:100960004AEC02F0416E4AEC02F0426E4AEC02F0B0
:10097000436E060E49EC02F0106E030E105C05E3A8
:10098000060EA96E000E4FEC02F0820E056E020EEE
:100990000C6E010E0E6EA9EC01F009E3CC0E8FEC8B
:1009A00001F0440E8FEC01F0A6EC01F000E3820EA2
:1009B000056E020E0C6E010E0E6EA9EC01F009E33D
:1009C000CC0E8FEC01F0440E8FEC01F0A6EC01F0A0
:1009D00000E3020E196E580E5DEC02F060EC33F08D
:1009E0000DDA8180000E49EC02F0456E0A0E455C7E
:1009F000D8B0456AC6EC39F0030E196EE80E5DEC0E
:100A000002F0558066EC10F0C2EC23F0010E196E76
:100A1000F40E5DEC02F045C020F0216A030E186E62
:100A2000196A29DE276E1DC028F0120E272449EC12
:100A300002F0CA6F45C020F0216A030E186E196AD1
:100A40001ADE276E1DC028F0130E272449EC02F091
:100A5000CB6F45C020F0216A030E186E196A0BDEB9
:100A6000276E1DC028F0140E272449EC02F0CC6F2D
:100A7000D896E6A9D886D8B684D055B081D055800E
:100A800055A203D06CEC11F003D080EC23F0558418
:100A9000D892E6A5D882D8B2E685D8A2E695D896AF
:100AA000E6A5D88607E4D892E6A3D882D8B2E68332
:100AB000D8A2E693FDEC39F0180ECA5D010ED8A459
:100AC000000E316E190ECA5D010ED8A4000E31124F
:100AD0001A0ECA5D010ED8A4000E3112180ECB5D9D
:100AE000010ED8A4000E3112190ECB5D010ED8A450
:100AF000000E31121A0ECB5D010ED8A4000E311279
:100B0000090ECC5D010ED8A4000E3112D8A4EDEC74
:100B100011F0130ECA5D010ED8A4000E316E140E32
:100B2000CA5D010ED8A4000E3112150ECA5D010E69
:100B3000D8A4000E3112160ECA5D010ED8A4000E04
:100B40003112130ECB5D010ED8A4000E3112140E1B
:100B5000CB5D010ED8A4000E3112150ECB5D010E37
:100B6000D8A4000E3112160ECB5D010ED8A4000ED3
:100B70003112010E81BCE86A3112D8A43FD94AD89B
:100B800016D055A014D05590050E49EC02F0106E09
:100B9000010E105C09E155A203D06CEC11F003D0FA
:100BA00080EC23F0558436D855B20DEC17F081B6A1
:100BB00089D0810E056E800E0C6E256A2368246A2A
:100BC000010E266E565028EC02F0566ED8B021EF7A
:100BD00024F0810E056E200E0C6E256A2368246AAF
:100BE000010E266E585028EC02F0586ED8B076EF01
:100BF00009F0810E056E100E0C6E256A2368246ABA
:100C0000010E266E595028EC02F0596ED8B06AEFEA
:100C100009F02ED781BC1ED0E631E8320EE3060E75
:100C200049EC02F0106E020E105C02E1DAD804D03A
:100C300086EC09F08BEC09F00CD0060E49EC02F0C2
:100C4000106E105202E0CDD804D086EC09F08BEC87
:100C500009F037D055A435D002EC3BF0CAC0C9F03A
:100C6000010EFE6FDFEC22F009EC3BF0CBC0C9F0C7
:100C7000020EFE6FDFEC22F0030EFE6F020ECC5D63
:100C8000D8B40EEC19F0030ECC5DD8B4B7EC1DF05F
:100C9000040ECC5DD8B4FEEC19F0050ECC5DD8B4D2
:100CA00011EC1BF0060ECC5DD8B401EC1BF0070E66
:100CB000CC5DD8B48BEC1BF0080ECC5DD8B400EC46
:100CC0001CF012009BD827EC11F04EEC21F0590ECD
:100CD000A96EE9514FEC02F0EA514FEC02F0EB51F2
:100CE0004FEC02F0EC514FEC02F0ED514FEC02F002
:100CF000EE514FEC02F0EF514FEC02F0F0514FEC9F
:100D000002F0650EA96E3A504FEC02F0660EA96E25
:100D10003B504FEC02F03C504FEC02F03D504FEC9A
:100D200002F03E504FEC02F06A0EA96E40504FECBC
:100D300002F041504FEC02F042504FEC02F04350B1
:100D40004FEC02F0010E49EC02F0446EB96BC16B3E
:100D500081805590445206E18290030E196EE80E90
:100D60005DEC02F0D896E6A9D8861FE455B01CD0F9
:100D7000558081AE06D042D886EC09F08BEC09F0A4
:100D800001D02FD8B92B060EB95D02E1010EC16F5B
:100D9000010EC15DD8B481903C0EB95D05E1B96B1F
:100DA000FF0E445CD8A0440602D055B0559081A6F1
:100DB00017D6010E81BEE86A316E010E81BAE86A6B
:100DC0003112010E81B8E86A3112010E81BCE86A65
:100DD000311204E0010EC15DD8B4B4D7BBD7030013
:100DE000FED702EC3BF0010EFE6F8BEC1BF009EC22
:100DF0003BF0020EFE6F00EC1CF01200D10EE5EC91
:100E000001F0000EE5EC01F0C9EC01F0466EC9EC12
:100E100001F0486EC9EC01F04A6EC9EC01F04C6E6D
:100E2000C9EC01F04D6EC9EC01F04F6EC7EC01F05A
:100E3000516E48C053F05CD853C049F04AC053F0DB
:100E400057D853C04BF04DC053F052D853C04EF05A
:100E50004FC053F04DD853C050F051C053F048D854
:100E600053C052F046A809D0D00EE5EC01F0070EB1
:100E7000E5EC01F0100EE3EC01F0120049C053F074
:100E80004CD853C048F04BC053F047D853C04AF039
:100E90004EC053F042D853C04DF050C053F03DD82F
:100EA00053C04FF052C053F038D853C051F0466A87
:100EB0001200D00EE5EC01F0000EE5EC01F046501A
:100EC000E5EC01F04850E5EC01F04A50E5EC01F0AA
:100ED0004C50E5EC01F04D50E5EC01F04F50E5ECE5
:100EE00001F05150E5EC01F0100EE3EC01F01200BE
:100EF0000F0E5314546E53380F0B536E53C020F023
:100F0000216A0A0E186E196A3BEC03F0276E1DC0A9
:100F100028F054502724536E120053C014F00A0EC8
:100F2000E0EC02F0546E54C020F0216A0A0E186EF4
:100F3000196A3BEC03F0276E1DC028F02750535E62
:100F40005438276E286EF00E27160F0E28162750DD
:100F500053261200466ADAD905EC0DF0BCEC39F0E4
:100F6000810E056E800E0C6E256A2368246A010EC0
:100F7000266E565028EC02F0566ED8B01AEF28F0C4
:100F8000810E056E400E0C6E256A2368246A010EE0
:100F9000266E575028EC02F0576E1FE2810E056E48
:100FA000200E0C6E256A2368246A010E266E5850A6
:100FB00028EC02F0586ED8B018D1810E056E100ED4
:100FC0000C6E256A2368246A010E266E595028EC9F
:100FD00002F0596ED8B015D1C1D798D908EC0DF0F0
:100FE000BCEC39F0810E056E400E0C6E256A23684C
:100FF000246A010E266E575028EC02F0576E2EE23E
:10100000810E056E800E0C6E256A2368246A010E1F
:10101000266E565028EC02F0566ED8B09BD7810E43
:10102000056E200E0C6E256A2368246A010E266E5A
:10103000585028EC02F0586ED8B0EED0810E056EF4
:10104000100E0C6E256A2368246A010E266E595014
:1010500028EC02F0596ED8B0EBD0C2D761D905ECBC
:101060000DF0BCEC39F0810E056E400E0C6E256A59
:101070002368246A010E266E575028EC02F0576E42
:101080002EE2810E056E800E0C6E256A2368246A9E
:10109000010E266E565028EC02F0566ED8B09DD741
:1010A000810E056E200E0C6E256A2368246A010EDF
:1010B000266E585028EC02F0586ED8B0C4D0810E7D
:1010C000056E100E0C6E256A2368246A010E266ECA
:1010D000595028EC02F0596ED8B0C1D0C2D720D9EF
:1010E00008EC0DF0BCEC39F0810E056E400E0C6E74
:1010F000256A2368246A010E266E575028EC02F0F8
:10110000576E2EE2810E056E800E0C6E256A2368E6
:10111000246A010E266E565028EC02F0566ED8B0A6
:101120009DD7810E056E200E0C6E256A2368246AF9
:10113000010E266E585028EC02F0586ED8B09BD0A5
:10114000810E056E100E0C6E256A2368246A010E4E
:10115000266E595028EC02F0596ED8B098D0C2D7FC
:10116000DFD812EC0DF0BCEC39F0810E056E400EAC
:101170000C6E256A2368246A010E266E575028ECEF
:1011800002F0576E2EE2810E056E800E0C6E256AFF
:101190002368246A010E266E565028EC02F0566E23
:1011A000D8B09DD7810E056E200E0C6E256A23687F
:1011B000246A010E266E585028EC02F0586ED8B002
:1011C00072D0810E056E100E0C6E256A2368246A9B
:1011D000010E266E595028EC02F0596ED8B06FD02F
:1011E000C2D74CDE66DE1AEF28F0170E4B5CD8A093
:1011F0004B2A44DE8BD805EC0DF0640E5CEC02F05B
:10120000A9D64B52D8A44B0639DE80D805EC0DF098
:10121000640E5CEC02F09ED63B0E495CD8A0492AD5
:101220002DDE74D808EC0DF0640E5CEC02F0D5D61F
:101230004952D8A4490622DE69D808EC0DF0640EA4
:101240005CEC02F0CAD61F0E4E5CD8A04E2A16DE09
:1012500067D805EC0DF0640E5CEC02F0FFD6020ED0
:101260004E5CD8B04E060ADE5BD805EC0DF0640E7D
:101270005CEC02F0F3D60C0E505CD8A0502AFEDDD8
:101280004FD808EC0DF0640E5CEC02F028D7020E8B
:10129000505CD8B05006F2DD43D808EC0DF0640E77
:1012A0005CEC02F01CD7630E525CD8A0522AE6DD3B
:1012B00037D812EC0DF0640E5CEC02F051D75252AC
:1012C000D8A45206DBDD2CD812EC0DF0640E5CECD9
:1012D00002F046D781BC04D0090E456E04EF05F03C
:1012E000090E455CD8A0452A04EF05F081BC03D067
:1012F000456A04EF05F04552D8A4450604EF05F011
:10130000A96A45504FEC02F004EF05F09AEC23F087
:10131000B8EC1EF0120009EC3BF0D4EC1EF0120009
:101320009AEC23F0D4EC1EF01200010EB96F558632
:1013300045C027F0286A27C020F028C021F0030EFE
:10134000186E196A3BEC03F0276E1DC028F0B951E6
:101350002726000E2822110E2724C96FC95149ECF7
:1013600002F0C96F030EB95D06E21B0EC95D02E310
:10137000010EC96F05D0090EC95D02E3010EC96FE8
:1013800055A6A7D255969AEC23F0C80E92EC00F021
:10139000A80E92EC00F0610E92EC00F0700E92EC50
:1013A00000F02E0E92EC00F0200E92EC00F0800E79
:1013B000016E010E0B6EB95133EC00F0030EB95DF6
:1013C000D8B0FBD1C90E92EC00F009EC3BF0D90E7D
:1013D00092EC00F0010EC95D12E1510E92EC00F0AA
:1013E000200E92EC00F0BC0E92EC00F0B80E92ECE5
:1013F00000F0BF0E92EC00F02E0E92EC00F0020E08
:10140000C95D12E1510E92EC00F0200E92EC00F05A
:10141000630E92EC00F0650E92EC00F0700E92EC10
:1014200000F02E0E92EC00F0030EC95D12E1510E99
:1014300092EC00F0200E92EC00F0B70E92EC00F06F
:10144000610E92EC00F0B40E92EC00F02E0E92ECD5
:1014500000F0040EC95D12E1510E92EC00F0200E76
:1014600092EC00F0BE0E92EC00F06F0E92EC00F0E9
:10147000040E92EC00F0B70E92EC00F0050EC95D80
:1014800012E14F0E92EC00F0B20E92EC00F02E0E34
:1014900092EC00F0E30E92EC00F0B30E92EC00F050
:1014A0002E0E92EC00F0060EC95D12E1250E92ECB4
:1014B00000F0200E92EC00F0E30E92EC00F0700EC3
:1014C00092EC00F06F0E92EC00F0630E92EC00F0E4
:1014D000070EC95D12E14B0E92EC00F0790E92EC12
:1014E00000F0BF0E92EC00F0200E92EC00F0B70E70
:1014F00092EC00F0BE0E92EC00F0080EC95D12E115
:10150000540E92EC00F0200E92EC00F0B30E92EC30
:1015100000F0BE0E92EC00F0700E92EC00F02E0E79
:1015200092EC00F0090EC95D12E1540E92EC00F04D
:10153000200E92EC00F0BD0E92EC00F0610E92ECE9
:1015400000F0BA0E92EC00F02E0E92EC00F00A0EB3
:10155000C95D12E1500E92EC00F0200E92EC00F00A
:10156000610E92EC00F0B20E92EC00F0630E92EC81
:1015700000F02E0E92EC00F00B0EC95D12E1740E1D
:1015800092EC00F0200E92EC00F0E30E92EC00F0F2
:10159000B30E92EC00F0B80E92EC00F0B40E92ECA8
:1015A00000F00C0EC95D12E1740E92EC00F0200EFA
:1015B00092EC00F0610E92EC00F0BF0E92EC00F0A5
:1015C000BC0E92EC00F02E0E92EC00F00D0EC95DF8
:1015D00006E1060EF76ECE0EF66E8AEC00F00E0EE9
:1015E000C95D06E1060EF76ED60EF66E8AEC00F0C7
:1015F0000F0EC95D12E1AC0E92EC00F0B30E92EC4E
:1016000000F0B80E92EC00F0E30E92EC00F0BA0E8F
:1016100092EC00F02E0E92EC00F0100EC95D12E17B
:10162000550E92EC00F0200E92EC00F0610E92EC60
:1016300000F0BA0E92EC00F0B20E92EC00F0200E28
:1016400092EC00F0110EC95D12E1200E92EC00F058
:10165000550E92EC00F0200E92EC00F0E00E92ECB1
:1016600000F04B0E92EC00F0200E92EC00F0120E07
:10167000C95D12E1500E92EC00F0580E92EC00F0B1
:10168000580E92EC00F0200E92EC00F0BA0E92ECA4
:1016900000F0700E92EC00F0130EC95D12E1AB0E7B
:1016A00092EC00F0610E92EC00F0630E92EC00F010
:1016B000200E92EC00F04B0E92EC00F0200E92EC1B
:1016C00000F0140EC95D12E1AB0E92EC00F0610E59
:1016D00092EC00F0630E92EC00F0200E92EC00F021
:1016E000A80E92EC00F0200E92EC00F0150EC95DF1
:1016F00012E1E00E92EC00F0610E92EC00F0BF0EF1
:1017000092EC00F0610E92EC00F0200E92EC00F0F2
:101710004B0E92EC00F0160EC95D12E1E00E92EC59
:1017200000F0610E92EC00F0BF0E92EC00F0610E42
:1017300092EC00F0200E92EC00F0A80E92EC00F07B
:10174000170EC95D12E14F0E92EC00F0E30E92EC21
:1017500000F06F0E92EC00F0BC0E92EC00F02E0E3A
:1017600092EC00F0200E92EC00F0180EC95D06E13C
:10177000060EF76EDE0EF66E8AEC00F0190EC95DED
:1017800012E14B0E92EC00F0790E92EC00F0BF0EDD
:1017900092EC00F0E00E92EC00F0BF0E92EC00F044
:1017A000BD0E92EC00F01A0EC95D06E1060EF76E52
:1017B000E60EF66E8AEC00F089D009EC3BF0D90E0B
:1017C00092EC00F0010EC95D06E1060EF76EEE0E1A
:1017D000F66E8AEC00F0020EC95D12E1500E92EC3A
:1017E00000F0650E92EC00F0B60E92EC00F0B80E30
:1017F00092EC00F0BC0E92EC00F0200E92EC00F0A7
:10180000030EC95D12E1500E92EC00F0580E92ECFE
:1018100000F0580E92EC00F0200E92EC00F0BA0EA0
:1018200092EC00F0700E92EC00F0040EC95D12E133
:10183000250E92EC00F0200E92EC00F0E30E92ECFC
:1018400000F0700E92EC00F06F0E92EC00F0630E60
:1018500092EC00F0050EC95D12E1740E92EC00F0FE
:10186000200E92EC00F0610E92EC00F0BF0E92ECB4
:1018700000F0BC0E92EC00F02E0E92EC00F0060E82
:10188000C95D12E1740E92EC00F0200E92EC00F0B3
:10189000E30E92EC00F0B30E92EC00F0B80E92EC76
:1018A00000F0B40E92EC00F0070EC95D06E1060EE2
:1018B000F76EF60EF66E8AEC00F0080EC95D06E1D2
:1018C000060EF76EFE0EF66E8AEC00F0DA0E92EC63
:1018D00000F0810E056E800E0C6E256A2368246A66
:1018E000010E266E565028EC02F0566E2FE2810E45
:1018F000056E400E0C6E256A2368246A010E266E62
:10190000575028EC02F0576E2BE2810E056E100E38
:101910000C6E256A2368246A010E266E595028EC45
:1019200002F0596ED8B046D0810E056E200E0C6EB6
:10193000256A2368246A010E266E585028EC02F0AE
:10194000586E15E2BCEC39F098EF09F05586010E9F
:10195000B95D03E121EF24F001D0B90798EF09F058
:101960005586030EB95DD8A0B92B98EF09F05586BE
:10197000020EC95DD8B0C907110E276E286A45C08E
:101980002BF02C6A2BC020F02CC021F0030E186E17
:10199000196A3BEC03F02B6E1DC02CF02B50272650
:1019A0002C502822B9512724A96EC9514FEC02F0BE
:1019B00098EF09F05586030EB95D05E21A0EC95D70
:1019C000D8A0C92B04D0080EC95DD8A0C92B110E10
:1019D000276E286A45C02BF02C6A2BC020F02CC043
:1019E00021F0030E186E196A3BEC03F02B6E1DC03C
:1019F0002CF02B5027262C502822B9512724A96ED1
:101A0000C9514FEC02F098EF09F009EC3BF013D00C
:101A100009EC3BF0200E92EC00F092EC00F092EC1E
:101A200000F009D009EC3BF0070EF76E060EF66EDB
:101A30008AEC00F000D0060E92EC00F0060E92EC5C
:101A400000F0120056EC12F08D51106E7F0E105CFB
:101A5000F9E08D51106E580E105CD8A4E1EF2AF019
:101A6000010EF36F558655A67CD055969AEC23F05F
:101A70008E51106E105233E1A80E92EC00F06F0EF2
:101A800092EC00F0BC0E92EC00F0B80E92EC00F07C
:101A9000BB0E92EC00F02E0E92EC00F0200E92ECB9
:101AA00000F0300E92EC00F009EC3BF03C0E92ECB2
:101AB00000F0200E92EC00F0200E92EC00F0B30E3D
:101AC00092EC00F0B80E92EC00F0780E92EC00F080
:101AD000690E92EC00F0E30E92EC00F042D0F3C0FD
:101AE00020F0216A030E186E196A3BEC03F0276E92
:101AF0001DC028F0020E2724B96F3C0E92EC00F0B6
:101B0000800E016E020E0B6EF35133EC00F02F0EBF
:101B100092EC00F092EC00F0020E0B6E8E5133EC62
:101B200000F03E0E92EC00F009EC3BF0200E92EC3F
:101B300000F0500E92EC00F0200E92EC00F0800EBF
:101B4000016E020E0B6E00EE8AF0B951EB501DECE7
:101B500000F0020E0B6EB92900EE8AF0EB501DEC7E
:101B600000F0BCEC39F0810E056E800E0C6E256A1B
:101B70002368246A010E266E565028EC02F0566E39
:101B80000FE2810E056E400E0C6E256A2368246AF2
:101B9000010E266E575028EC02F0576E07E263D70D
:101BA000F307F353D8B4E1EF2AF05CD7F32B0F0E11
:101BB000F35D010ED8A4000E316E8E51106EF3C08D
:101BC00014F0105006EC00F0311202E0010EF36F39
:101BD00049D7F16BF46B080EF45DD8B064D0F453C0
:101BE00002E1E9C0E8F0010EF45D02E1EAC0E8F0CC
:101BF000020EF45D02E1EBC0E8F0030EF45D02E1D9
:101C0000ECC0E8F0040EF45D02E1EDC0E8F0050E72
:101C1000F45D02E1EEC0E8F0060EF45D02E1EFC013
:101C2000E8F0070EF45D02E1F0C0E8F0F56B080E95
:101C3000F55D36E2F55303E1E687E8A1E697010E8C
:101C4000F55D03E1E687E8A3E697020EF55D03E1A3
:101C5000E687E8A5E697030EF55D03E1E687E8A7CA
:101C6000E697040EF55D03E1E687E8A9E697050E21
:101C7000F55D03E1E687E8ABE697060EF55D03E167
:101C8000E687E8ADE697070EF55D03E1E687E8AF86
:101C9000E697D896E6A7D886D8A6F12BF52BC7E10C
:101CA000F42BD8A498D7010EF36F558655A658D0BB
:101CB00055969AEC23F0F15333E1A80E92EC00F024
:101CC0006F0E92EC00F0BC0E92EC00F0B80E92ECAD
:101CD00000F0BB0E92EC00F02E0E92EC00F0200E05
:101CE00092EC00F0300E92EC00F009EC3BF03C0E70
:101CF00092EC00F0200E92EC00F0200E92EC00F03E
:101D0000B30E92EC00F0B80E92EC00F0780E92EC6C
:101D100000F0690E92EC00F0E30E92EC00F020D09F
:101D20004BD83C0E92EC00F0800E016E020E0B6E52
:101D3000F35133EC00F02F0E92EC00F092EC00F037
:101D4000020E0B6EF15133EC00F03E0E92EC00F0FF
:101D500009EC3BF0070EF76E0E0EF66E8AEC00F003
:101D6000BCEC39F0810E056E800E0C6E256A23687E
:101D7000246A010E266E565028EC02F0566E0FE2D1
:101D8000810E056E400E0C6E256A2368246A010ED2
:101D9000266E575028EC02F0576E07E287D7F307FC
:101DA000F353D8B4E1EF2AF080D7F32BF351F15D70
:101DB00002E2010EF36F79D7F26BF46B080EF45D5B
:101DC000D8B06AD0F45302E1E9C0E8F0010EF45D46
:101DD00002E1EAC0E8F0020EF45D02E1EBC0E8F0D7
:101DE000030EF45D02E1ECC0E8F0040EF45D02E1E4
:101DF000EDC0E8F0050EF45D02E1EEC0E8F0060E7D
:101E0000F45D02E1EFC0E8F0070EF45D02E1F0C01E
:101E1000E8F0F56B080EF55D39E2F55303E1E6876E
:101E2000E8A1E697010EF55D03E1E687E8A3E697F2
:101E3000020EF55D03E1E687E8A5E697030EF55D82
:101E400003E1E687E8A7E697040EF55D03E1E68780
:101E5000E8A9E697050EF55D03E1E687E8ABE697AE
:101E6000060EF55D03E1E687E8ADE697070EF55D42
:101E700003E1E687E8AFE697D896E6A7D886D8A626
:101E8000F22BF251F35D02E0F52BC4E1F251F35D68
:101E900003E0F42BD8A492D71200F16BF46B040E7C
:101EA000F45DD8B050D0F45302E15F50E86F010EFA
:101EB000F45D02E16050E86F020EF45D02E16150F2
:101EC000E86F030EF45D02E16250E86FF56B080EF7
:101ED000F55D36E2F55303E1E687E8A1E697010EEA
:101EE000F55D03E1E687E8A3E697020EF55D03E101
:101EF000E687E8A5E697030EF55D03E1E687E8A728
:101F0000E697040EF55D03E1E687E8A9E697050E7E
:101F1000F55D03E1E687E8ABE697060EF55D03E1C4
:101F2000E687E8ADE697070EF55D03E1E687E8AFE3
:101F3000E697D896E6A7D886D8A6F12BF52BC7E169
:101F4000F42BD8A4ACD7010EF36F558655A635D027
:101F500055969AEC23F05DD83C0E92EC00F0800E82
:101F6000016E020E0B6EF35133EC00F02F0E92EC6B
:101F700000F092EC00F0020E0B6EF15133EC00F029
:101F80003E0E92EC00F009EC3BF04B0E92EC00F0B0
:101F90004D0E92EC00F0A80E92EC00F0200E92ECA8
:101FA00000F0800E016E020E0B6EF45133EC00F067
:101FB000020E0B6EF55133EC00F0BCEC39F0810EE3
:101FC000056E800E0C6E256A2368246A010E266E4B
:101FD000565028EC02F0566E0FE2810E056E400E50
:101FE0000C6E256A2368246A010E266E575028EC71
:101FF00002F0576E07E2AAD7F307F353D8B4E1EF24
:102000002AF0A3D7F32BF351F15D02E2010EF36F37
:102010009CD7F26BF46B040EF45DD8B056D0F45339
:1020200002E15F50E86F010EF45D02E16050E86F7D
:10203000020EF45D02E16150E86F030EF45D02E10F
:102040006250E86FF56B080EF55D39E2F55303E178
:10205000E687E8A1E697010EF55D03E1E687E8A3D0
:10206000E697020EF55D03E1E687E8A5E697030E25
:10207000F55D03E1E687E8A7E697040EF55D03E169
:10208000E687E8A9E697050EF55D03E1E687E8AB8C
:10209000E697060EF55D03E1E687E8ADE697070EE5
:1020A000F55D03E1E687E8AFE697D896E6A7D88620
:1020B000D8A6F22BF251F35D02E0F52BC4E1F25108
:1020C000F35D03E0F42BD8A4A6D7120081B662EF2B
:1020D00006F080EC23F0810E056E800E0C6E256AF2
:1020E0002368246A010E266E565028EC02F0566EC4
:1020F000D8B0ABD09AEC23F0070EF76E180EF66E40
:102100008AEC00F009EC3BF0070EF76E200EF66E3D
:102110008AEC00F0828C010E196E2C0E5DEC02F040
:10212000829C610E156EA80E6AEC02F0828C5D0E28
:10213000156EC00E6AEC02F0820E056E400E0C6E3B
:102140004C0E236E246A086A096A200E016E810E05
:1021500020EC01F0100E20EC01F0F10E20EC01F06B
:10216000810E20EC01F0030E20EC01F0820E056ED2
:10217000800E0C6E4C0E236E246ABC0E086E020E8E
:10218000096E106AD880DEEC00F009E300EE5AF028
:10219000105018C0EBFF102A10500708F3E15D50F3
:1021A000106EC10E105C05E155825E50E76F1200A3
:1021B0004CD09AEC23F0800E016E020E0B6E5A503A
:1021C0001DEC00F0020E0B6E5B501DEC00F0020ED9
:1021D0000B6E5C501DEC00F0020E0B6E5D501DECA2
:1021E00000F009EC3BF0800E016E020E0B6E5E50AB
:1021F0001DEC00F0020E0B6E5F501DEC00F0020EA5
:102200000B6E60501DEC00F05592820E056E400E74
:102210000C6E4C0E236E246A086A096A200E016E49
:10222000810E20EC01F0100E20EC01F0F10E20ECFC
:1022300001F0820E20EC01F0040E20EC01F0030E00
:10224000196EE80E5DEC02F041D755921200810E36
:10225000056E800E0C6E256A2368246A010E266EB8
:10226000565028EC02F0566E35E29AEC23F0530EED
:1022700092EC00F0740E92EC00F06F0E92EC00F015
:10228000700E92EC00F009EC3BF0070EF76E2A0E90
:10229000F66E8AEC00F0820E056E400E0C6E4C0E4F
:1022A000236E246A086A096A200E016E810E20ECF2
:1022B00001F0100E20EC01F0F10E20EC01F0820E86
:1022C00020EC01F0040E20EC01F0010E196EF40E6A
:1022D0005DEC02F05592120080EC23F0820E056E48
:1022E000400E0C6E4C0E236E246A086A096A200E9A
:1022F000016E820E20EC01F0100E20EC01F0F10EC8
:1023000020EC01F0210E20EC01F0010E20EC01F098
:10231000A50E20EC01F06B0EE75D010ED8A4000EB7
:10232000316E080E49EC02F0106E020E105CD8A45B
:10233000010E311624E0820E056E800E0C6E4C0EDE
:10234000236E246A2C0E086E010E096E106AD88066
:10235000DEEC00F03AE300EE5AF0105018C0EBFF4C
:10236000102A10503008F3E1090E0B6E0B50D88084
:1023700005E0DEEC00F029E30B06F8D719D0820E59
:10238000056E800E0C6E4C0E236E246A2C0E086EA9
:10239000010E096E106AD880DEEC00F016E300EE44
:1023A0005AF0105018C0EBFF102A10502F08F3E11C
:1023B0005D50106E610E105C05E15584BA6B32D928
:1023C000120003D05594BA6B12005594BA2B0A0E22
:1023D000BA5D02E13CDF7ADE1200820E056E400E2D
:1023E0000C6E4C0E236E246A086A096A200E016E78
:1023F000820E20EC01F0100E20EC01F0F10E20EC2A
:1024000001F0210E20EC01F0E10E20EC01F0850E30
:1024100020EC01F0820E056E800E0C6E4C0E236EC9
:10242000246A580E086E020E096E260E0B6E0B50B3
:10243000D88005E0DEEC00F038E30B06F8D7DEECE0
:1024400000F033E3396EDEEC00F02FE3386E020E5D
:102450000B6E0B50D88005E0DEEC00F026E30B0697
:10246000F8D7DEEC00F021E3356EDEEC00F01DE382
:10247000346E060E0B6E0B50D88005E0DEEC00F0DB
:1024800014E30B06F8D7DEEC00F00FE3376EDEEC5A
:1024900000F00BE3366E470E0B6E0B50D88005E054
:1024A000DEEC00F002E30B06F8D712008DEC23F00F
:1024B000820E056E400E0C6E4C0E236E246A086A66
:1024C000096A200E016E840E20EC01F0100E20EC43
:1024D00001F0F10E20EC01F0180E20EC01F0000EDE
:1024E00020EC01F0FF0E20EC01F0000E20EC01F0DA
:1024F0009C0E20EC01F0820E056E800E0C6E4C0ED0
:10250000236E246AF40E086E010E096E106AD880DC
:10251000DEEC00F009E300EE8AF0105018C0EBFF8B
:10252000102A10502F08F3E11200820E056E400EA3
:102530000C6E4C0E236E246A086A096A200E016E26
:10254000820E20EC01F0100E20EC01F0F10E20ECD8
:1025500001F03E0E20EC01F0020E20EC01F0C30E63
:1025600020EC01F01200820E056E400E0C6E4C0E37
:10257000236E246A086A096A200E016E830E20EC1D
:1025800001F0100E20EC01F0F10E20EC01F0140E21
:1025900020EC01F0FF0E20EC01F0000E20EC01F029
:1025A000970E20EC01F0820E056E800E0C6E4C0E24
:1025B000236E246ABC0E086E020E096E070E0B6EA7
:1025C0000B50D88005E0DEEC00F002E30B06F8D7F4
:1025D000640E5CEC02F022EF0DF0590EA96E000EB5
:1025E0004FEC02F0000E4FEC02F0000E4FEC02F048
:1025F000000E4FEC02F0000E4FEC02F0000E4FEC1C
:1026000002F0000E4FEC02F0000E4FEC02F0E96B0E
:10261000EA6BEB6BEC6BED6BEE6BEF6BF06B02D878
:10262000E9EF0DF06350106E1050E9136450106E16
:102630001050EA136550106E1050EB136650106E78
:102640001050EC136750106E1050ED136850106E60
:102650001050EE136950106E1050EF136A50106E48
:102660001050F013120080EC23F0010EFC5D04E129
:10267000F90E466E420E486E020EFC5D04E1180E25
:10268000466E610E486E030EFC5D04E11A0E466E46
:10269000630E486E080EFC5D06E1F80E466EF70EFE
:1026A000476E410E486E090EFC5D06E1080E466E4F
:1026B000070E476E510E486E0A0EFC5D06E1FB0EDA
:1026C000466EFA0E476E440E486E820E056E400E40
:1026D0000C6E4C0E236E246A086A096A200E016E85
:1026E000850E20EC01F0100E20EC01F0F10E20EC34
:1026F00001F0300E20EC01F0485020EC01F0010E0A
:1027000020EC01F0000E20EC01F0000E20EC01F0B6
:10271000465020EC01F0820E056E800E0C6E4C0EC1
:10272000236E246A580E086E020E096E106AD88055
:10273000DEEC00F00DE300EE5AF0105018C0EBFF95
:10274000102A10500908F3E16050C86F6150C76F3C
:1027500012005586E69187DF55A6A7D055969AECCC
:1027600023F0010EFC5D18E14F0E92EC00F0B20E6A
:1027700092EC00F0650E92EC00F0700E92EC00F01E
:10278000BF0E92EC00F0580E92EC00F0580E92EC56
:1027900000F03E0E92EC00F0020EFC5D18E1A90E76
:1027A00092EC00F0630E92EC00F0BF0E92EC00F0A1
:1027B000470E92EC00F0300E92EC00F0580E92ECC6
:1027C00000F0580E92EC00F03E0E92EC00F0030E7A
:1027D000FC5D18E1A90E92EC00F0630E92EC00F0A3
:1027E000BF0E92EC00F02E0E92EC00F0470E92EC31
:1027F00000F0300E92EC00F0420E92EC00F03E0E33
:1028000092EC00F0080EFC5D18E1A90E92EC00F0CD
:10281000BE0E92EC00F0700E92EC00F02E0E92ECD8
:1028200000F0500E92EC00F0580E92EC00F0580EB2
:1028300092EC00F03E0E92EC00F0090EFC5D18E107
:10284000410E92EC00F0E30E92EC00F0630E92EC7D
:1028500000F06F0E92EC00F0700E92EC00F0B20EF1
:1028600092EC00F02E0E92EC00F03E0E92EC00F096
:102870000A0EFC5D18E14B0E92EC00F0790E92EC22
:1028800000F0BF0E92EC00F0A40E92EC00F0610E8E
:1028900092EC00F0BE0E92EC00F02E0E92EC00F0E6
:1028A0003E0E92EC00F04EEC39F055B24FEC33F0A6
:1028B00081A603D04CD862EF06F0640E5CEC02F007
:1028C000810E056E400E0C6E256A2368246A010E87
:1028D000266E575028EC02F0576ED8B0A9EF38F0AA
:1028E000810E056E800E0C6E256A2368246A010E27
:1028F000266E565028EC02F0566E25E2040EFC5D62
:102900000FE2810E056E200E0C6E256A2368246A84
:10291000010E266E585028EC02F0586ED8B0C6D082
:10292000040EFC5D0FE2810E056E100E0C6E256A22
:102930002368246A010E266E595028EC02F0596E65
:10294000D8B0CAD009D703D85586D1EF2CF0820E63
:10295000056E400E0C6E4C0E236E246A086A096ADE
:10296000200E016E850E20EC01F0100E20EC01F01F
:10297000F10E20EC01F0300E20EC01F0485020EC7C
:1029800001F0000E20EC01F0000E20EC01F0000E32
:1029900020EC01F0475020EC01F0120080EC23F015
:1029A000C8C0C1F0C7C0C2F0010EFC5D04E1420E18
:1029B000486E080E4A6E020EFC5D06E1690E462660
:1029C000610E486E080E4A6E030EFC5D04E1630E54
:1029D000486E080E4A6E080EFC5D04E1410E486E1A
:1029E000070E4A6E090EFC5D04E1510E486E070E9B
:1029F0004A6E0A0EFC5D04E1440E486E070E4A6EF4
:102A0000B60E276E286A48502726000E28224A5004
:102A10002726000E2822C1512726000E2822C25147
:102A20002724466E820E056E400E0C6E4C0E236EF1
:102A3000246A086A096A200E016E850E20EC01F0F6
:102A4000100E20EC01F0F10E20EC01F0300E20EC25
:102A500001F0485020EC01F04A5020EC01F0C15147
:102A600020EC01F0C25120EC01F0465020EC01F0C6
:102A7000820E056E800E0C6E4C0E236E246A580E6C
:102A8000086E020E096E106AD880DEEC00F00DE3CD
:102A900000EE5AF0105018C0EBFF102A1050090831
:102AA000F3E16050C86F6150C76F1200558681BC5A
:102AB00005D00A0EC727000EC82302D0C74BC82B6B
:102AC0006DDFE631D8A048D6E63106E3D896E6A118
:102AD000D886D8A6A9EF38F0558681BC0AD0C8534D
:102AE00003E10A0EC75D04E30A0EC75F000EC85B70
:102AF00007D0C75302E1C85303E0C707000EC85B05
:102B00004DDFE631D8A028D6E63106E3D896E6A117
:102B1000D886D8A6A9EF38F080EC23F0820E056E97
:102B2000400E0C6E4C0E236E246A086A096A200E51
:102B3000016E820E20EC01F0100E20EC01F0F10E7F
:102B400020EC01F0210E20EC01F0E20E20EC01F06F
:102B5000860E20EC01F0820E056E800E0C6E4C0E7F
:102B6000236E246A580E086E020E096E106AD88011
:102B7000DEEC00F009E300EE5AF0105018C0EBFF55
:102B8000102A10502608F3E11200558655A61AD0D7
:102B900055969AEC23F0A80E92EC00F06F0E92EC92
:102BA00000F0C00E92EC00F0610E92EC00F0BF0E4F
:102BB00092EC00F0B80E92EC00F03F0E92EC00F0B8
:102BC000E8EC3AF0BCEC39F0810E056E800E0C6E2C
:102BD000256A2368246A010E266E565028EC02F0FE
:102BE000566ED8B0CFEF2CF0810E056E200E0C6E15
:102BF000256A2368246A010E266E585028EC02F0DC
:102C0000586E11E2810E056E100E0C6E256A236857
:102C1000246A010E266E595028EC02F0596ED8B085
:102C2000CFEF2CF0B3D780EC23F09AEC23F0070E13
:102C3000F76E340EF66E8AEC00F0030E196EE80E95
:102C40005DEC02F0A2D7558655A61DD055969AEC9C
:102C500023F0A80E92EC00F0700E92EC00F0B80E8B
:102C600092EC00F0B90E92EC00F0BD0E92EC00F088
:102C7000C70E92EC00F0BF0E92EC00F0B80E92EC92
:102C800000F0E8EC3AF081B662EF06F055B244DFAE
:102C9000640E5CEC02F0810E056E800E0C6E256AEF
:102CA0002368246A010E266E565028EC02F0566EF8
:102CB000D8B06BD7810E056E200E0C6E256A236886
:102CC000246A010E266E585028EC02F0586E10E26D
:102CD000810E056E100E0C6E256A2368246A010EA3
:102CE000266E595028EC02F0596ED8B04ED7ACD7AA
:102CF00080EC23F0820E056E400E0C6E4C0E236E9F
:102D0000246A086A096A200E016E820E20EC01F026
:102D1000100E20EC01F0F10E20EC01F0310E20EC51
:102D200001F0110E20EC01F0C50E20EC01F0820E36
:102D3000056E800E0C6E4C0E236E246A580E086EC3
:102D4000020E096E106AD880DEEC00F035E300EE6A
:102D50005AF0105018C0EBFF102A10500608F3E18B
:102D60009AEC23F05D50106E710E105C010ED8A429
:102D7000000E316E5E50106E010E105C010ED8A474
:102D8000000E311619E0A90E92EC00F0630E92ECE1
:102D900000F0BE0E92EC00F0690E92EC00F0C10E55
:102DA00092EC00F0BD0E92EC00F06F0E92EC00F091
:102DB00014D8CFEF2CF011D0200E92EC00F0200EA2
:102DC00092EC00F0200E92EC00F0480E92EC00F035
:102DD000650E92EC00F001D8D8D609EC3BF0BE0E9F
:102DE00092EC00F0700E92EC00F0B80E92EC00F055
:102DF000B90E92EC00F0BD0E92EC00F0C70E92EC12
:102E000000F0BF0E92EC00F06F0E92EC00F0030E9B
:102E1000196EE80E5DEC02F01200D86BD76BD66B22
:102E2000D56B820E056E400E0C6E4C0E236E246A1E
:102E3000086A096A200E016E820E20EC01F0100E65
:102E400020EC01F0F10E20EC01F0210E20EC01F05D
:102E5000F30E20EC01F0970E20EC01F06B0EE75D15
:102E6000010ED8A4000E316E080E49EC02F0106E6F
:102E7000020E105CD8A4010E3116D8B474D0820EA4
:102E8000056E800E0C6E4C0E236E246A580E086E72
:102E9000020E096E0A0E0B6E0B50D88006E0DEECB7
:102EA00000F0D8A0C5D00B06F7D7DEEC00F0D8A014
:102EB000BFD0D86FDEEC00F0D8A0BAD0D76FDEEC70
:102EC00000F0D8A0B5D0D66FDEEC00F0D8A0B0D01E
:102ED000D56F080E0B6E0B50D88006E0DEEC00F0CC
:102EE000D8A0A6D00B06F7D7DEEC00F0D8A0A0D073
:102EF000E06FDEEC00F0D8A09BD0DF6FDEEC00F0DE
:102F0000D8A096D0DE6FDEEC00F0D8A091D0DD6FB7
:102F1000200E0B6E0B50D88006E0DEEC00F0D8A03F
:102F200087D00B06F7D7DEEC00F0D8A081D0E46F95
:102F3000DEEC00F0D8A07CD0E36FDEEC00F0D8A08F
:102F400077D0E26FDEEC00F0D8A072D0E16F010E16
:102F50000B6E0B50D88006E0DEEC00F0D8A068D0F5
:102F60000B06F7D765D0820E056E800E0C6E4C0EE8
:102F7000236E246A580E086E020E096E0B0E0B6E3D
:102F80000B50D88006E0DEEC00F0D8A051D00B0644
:102F9000F7D7DEEC00F0D8A04BD0D86FDEEC00F015
:102FA00047E3D76FDEEC00F043E3D66FDEEC00F0D2
:102FB0003FE3D56F080E0B6E0B50D88005E0DEECBA
:102FC00000F036E30B06F8D7DEEC00F031E3E06FFB
:102FD000DEEC00F02DE3DF6FDEEC00F029E3DE6FC6
:102FE000DEEC00F025E3DD6F240E0B6E0B50D88075
:102FF00005E0DEEC00F01CE30B06F8D7DEEC00F099
:1030000017E3E46FDEEC00F013E3E36FDEEC00F0B7
:103010000FE3E26FDEEC00F00BE3E16F050E0B6EE9
:103020000B50D88005E0DEEC00F002E30B06F8D789
:103030001200020E49EC02F0466E7550BE6F7650DB
:10304000BD6F6F50C06F7050BF6FBDC020F0BEC06D
:1030500021F0BFC018F0C0C019F03BEC03F0BB6F0B
:103060001DC0BCF0030E196EE80ED2EC02F0C36F67
:1030700015C0C4F046C020F0216AC3C018F0C4C017
:1030800019F03BEC03F0BB6F1DC0BCF0030E196ED2
:10309000E80ED2EC02F0BB6F15C0BCF0030E49EC99
:1030A00002F0466E010E465C0CE0BBC020F0BCC0D6
:1030B00021F0020E186E196A3BEC03F0BB6F1DC0C5
:1030C000BCF0BBC020F0BCC021F0020E186E196A23
:1030D0003BEC03F0BB6F1DC0BCF08151106E060EBF
:1030E000105CD8A069D0BBC020F0BCC021F0640E39
:1030F000186E196A3BEC03F0BB6F1DC0BCF0815128
:10310000D1EC02F0BB6F15C0BCF0BBC014F0BCC06A
:1031100015F00A0E186E196AE3EC02F01CC010F0EC
:103120001DC011F0115203E1060E105C04E30A0EFB
:10313000BB27000EBC23BBC014F0BCC015F00A0EA8
:10314000186E196AE3EC02F0BB6F15C0BCF0BBC08F
:1031500014F0BCC015F00A0E186E196AE3EC02F008
:10316000C16FBBC014F0BCC015F00A0E186E196A0E
:10317000E3EC02F01CC0C2F00A0EC15D03E2200EB7
:1031800092EC00F0800E016EC15132EC00F02C0E7A
:1031900092EC00F0010E0B6EC25133EC00F0010E08
:1031A00092EC00F0020E92EC00F0BA0E92EC00F0FD
:1031B000BC0E92EC00F031D0BBC014F0BCC015F0D6
:1031C000640E186E196AE3EC02F0C16FBBC014F014
:1031D000BCC015F0640E186E196AE3EC02F01CC056
:1031E000C2F00A0EC15D03E2200E92EC00F0800EE8
:1031F000016EC15132EC00F02C0E92EC00F0020E88
:103200000B6EC25133EC00F0BB0E92EC00F02F0EAF
:1032100092EC00F0B40E92EC00F01200FE0E92EC74
:1032200000F0C00E92EC00F0010E446E070E445CFC
:1032300008E2FE0E92EC00F0140E92EC00F0442A2C
:10324000F5E16B50446E6C50B96FD896B9A7D8862B
:1032500007E4E00E92EC00F0540E92EC00F0120045
:10326000B935E83607E3A80E92EC00F0500E92EC68
:1032700000F01200E86A44B2010E316EE86A44B60A
:10328000010E31121AE0D896B9A5D88607E4450E8A
:1032900092EC00F0520E92EC00F00ED044A607D053
:1032A000A80E92EC00F0580E92EC00F005D0580EEB
:1032B00092EC00F092EC00F032D0E86A44B0010EDB
:1032C000316EE86A44B4010E311207E0A80E92ECA8
:1032D00000F0540E92EC00F022D044AE07D0500E15
:1032E00092EC00F0A80E92EC00F019D044B017D088
:1032F0006F50106E10C014F0000E06EC00F0316E2E
:103300007050106E10C014F0000E06EC00F0311278
:1033100006E0500E92EC00F0580E92EC00F0120015
:103320006F50BC6F7050BB6F030EBC5DE80ED8B41D
:10333000BB5D03E2200E92EC00F0BC5306E1640E8C
:10334000BB5D03E2200E92EC00F0BC5306E10A0ED6
:10335000BB5D03E2200E92EC00F0800E016E0B6A62
:10336000BBC01CF0BCC01DF035EC00F06F0E92EC41
:1033700000F0B20E92EC00F02F0E92EC00F0780EFE
:1033800092EC00F0120060D8BBC014F0BCC015F085
:103390000A0E186E196AE3EC02F01CC0C2F0640E4B
:1033A000C15D0CE3200E92EC00F0800E016EC15165
:1033B00032EC00F0250E92EC00F01FD00A0EC15D39
:1033C00003E2200E92EC00F0800E016EC15132EC4F
:1033D00000F02C0E92EC00F0010E0B6EC25133EC9B
:1033E00000F0250E92EC00F0200E92EC00F0E30EBF
:1033F00092EC00F0700E92EC00F0120025D8FE0E58
:1034000092EC00F0C00E92EC00F0010E446E070E3C
:10341000445C08E2FE0E92EC00F0140E92EC00F018
:10342000442AF5E1640EC15D08E2800E016E020ED1
:103430000B6EC15133EC00F006D04D0E92EC00F053
:10344000580E92EC00F012007150BC6F7250BB6FBE
:10345000BBC014F0BCC015F00A0E186E196AE3EC7C
:1034600002F0C16F12007350BC6F7450BB6FBBC0D1
:1034700014F0BCC015F00A0E186E196AE3EC02F0E5
:10348000C16FBBC014F0BCC015F00A0E186E196AEB
:10349000E3EC02F01CC0C2F0FE5309E04B0E92ECCC
:1034A00000F0B70E92EC00F0200E92EC00F00A0E45
:1034B000C15D03E2200E92EC00F0800E016EC1515E
:1034C00032EC00F02C0E92EC00F0010E0B6EC251AB
:1034D00033EC00F0FE5303E0000E92EC00F012001B
:1034E00034C014F035C015F00A0E186E196AE3ECFA
:1034F00002F0C16F34C014F035C015F00A0E186E1A
:10350000196AE3EC02F01CC0C2F0E00E92EC00F08D
:10351000BF0E92EC00F02D0E92EC00F00A0EC15D91
:1035200003E2200E92EC00F0800E016EC15132ECED
:1035300000F02C0E92EC00F0010E0B6EC25133EC39
:1035400000F0000E92EC00F012007550BC6F765047
:10355000BB6FBBC014F0BCC015F0640E186E196AC6
:10356000E3EC02F0C16FBBC014F0BCC015F0640EF8
:10357000186E196AE3EC02F01CC0C2F0FE530DE0B5
:10358000540E92EC00F0B30E92EC00F0BE0E92ECF2
:1035900000F0200E92EC00F006D00A0EC15D03E2AE
:1035A000200E92EC00F0800E016EC15132EC00F062
:1035B0002C0E92EC00F0020E0B6EC25133EC00F0B8
:1035C00012007950BC6F7A50BB6FFE530FE0500E63
:1035D00092EC00F0610E92EC00F0B20E92EC00F072
:1035E000630E92EC00F0200E92EC00F0800E016E63
:1035F000030E0B6EBBC01CF0BCC01DF035EC00F020
:103600001200030EFE5D09E2740E92EC00F0770EDC
:1036100092EC00F0200E92EC00F013D87B50C16FBA
:1036200027D0030EFE5D09E2740E92EC00F0610EED
:1036300092EC00F0200E92EC00F003D87C50C16FA9
:1036400017D0030EFE5D13E1FE0E92EC00F0C00EEB
:1036500092EC00F0010E446E060E445C08E2FE0E91
:1036600092EC00F0140E92EC00F0442AF5E1120006
:10367000280EC15D28E3D80EC125106E116AFF0E19
:103680001122115206E1640E105C03E2200E92EC4E
:1036900000F0D80EC125106E116AFF0E11221152D2
:1036A00006E10A0E105C03E2200E92EC00F0800EA0
:1036B000016E0B6AD80EC1251C6E1D6AFF0E1D22FD
:1036C00035EC00F01ED0C1512808106E000ED8A0B5
:1036D000FF0F116E115206E10A0E105C03E2200E7C
:1036E00092EC00F0070E92EC00F0800E016E0B6A77
:1036F000C15128081C6E000ED8A0FF0F1D6E35ECBE
:1037000000F0030EFE5D06E2000E92EC00F0430EA8
:1037100092EC00F012000101006B559E820E056EC6
:10372000020E0C6E010E0E6EA9EC01F00001D8A085
:10373000A2D1CC0E8FEC01F0440E8FEC01F0A6EC80
:1037400001F0D8A098D1820E056E020E0C6E040E08
:103750000E6EA9EC01F0D8A08ED170EC01F0106EC5
:10376000A6EC01F0D8A087D1105209E00101002B8E
:10377000640E005D000102E1558E01D0E4D7820E97
:10378000056E020E0C6E010E0E6EA9EC01F0D8A0B3
:1037900072D1CC0E8FEC01F0BE0E8FEC01F0A6ECD6
:1037A00001F0D8A068D1820E056E020E0C6E0E6E6E
:1037B000A9EC01F0D8A05FD170EC01F0BB6F70EC08
:1037C00001F0BC6F70EC01F0E56F70EC01F0E56F9B
:1037D00070EC01F0C16FA6EC01F0D8A04CD1558C73
:1037E000BCAF559C030EFE5D09E2740E92EC00F036
:1037F000690E92EC00F06E0E92EC00F076D812009A
:103800000101006B559E820E056E020E0C6E010EBC
:103810000E6EA9EC01F00001D8A02FD1CC0E8FECD8
:1038200001F0440E8FEC01F0A6EC01F0D8A025D1F8
:10383000820E056E020E0C6E040E0E6EA9EC01F0E7
:10384000D8A01BD170EC01F0106EA6EC01F0D8A04E
:1038500014D1105209E00101002B640E005D00013B
:1038600002E1558E01D0E4D7820E056E020E0C6E79
:10387000010E0E6EA9EC01F0D8A0FFD0CC0E8FEC9B
:1038800001F0BE0E8FEC01F0A6EC01F0D8A0F5D04F
:10389000820E056E020E0C6E0E6EA9EC01F0D8A021
:1038A000ECD070EC01F0BB6F70EC01F0BC6F70EC11
:1038B00001F0E56F70EC01F0E56F70EC01F0C16FA5
:1038C000A6EC01F0D8A0D9D0558CBCAF559C030E06
:1038D000FE5D09E2740E92EC00F0650E92EC00F0D1
:1038E000780E92EC00F001D81200030EFE5D13E199
:1038F000FE0E92EC00F0C00E92EC00F0010E446E51
:10390000060E445C08E2FE0E92EC00F0140E92ECFF
:1039100000F0442AF5E155BE73D055BC37D0BBC08A
:1039200027F0BCC028F027C020F028C021F00A0EE4
:10393000186E196A3BEC03F0276E1DC028F0040EC8
:10394000D89028322732E82EFBD727C014F028C0A1
:1039500015F00A0E186E196AE3EC02F01CC0C1F0F3
:10396000BC33BB33BC33BB33BC33BB33BC33BB33E3
:103970000F0EBC17BC5306E10A0EBB5D03E2200E1E
:1039800092EC00F0200E92EC00F03AD0BB1FBC1F6E
:10399000BBC027F0BCC028F0274A282A27C020F047
:1039A00028C021F00A0E186E196A3BEC03F0276E4E
:1039B0001DC028F0040ED89028322732E82EFBD7FD
:1039C00027C014F028C015F00A0E186E196AE3EC2F
:1039D00002F01CC0C1F0BC33BB33BC33BB33BC33BF
:1039E000BB33BC33BB330F0EBC17BC5306E10A0E0E
:1039F000BB5D03E2200E92EC00F0070E92EC00F0AB
:103A0000030EFE5D1FE255BE10D0800E016E0B6AE4
:103A1000BBC01CF0BCC01DF035EC00F02C0E92ECCD
:103A200000F0C15132EC00F00DD0200E92EC00F00D
:103A300092EC00F0450E92EC00F0720E92EC00F069
:103A400092EC00F0030EFE5D15E155BE0AD0800E2B
:103A5000016E0B6ABBC01CF0BCC01DF035EC00F061
:103A600009D0200E92EC00F0450E92EC00F0720EA0
:103A700092EC00F01200558EB2D6558E25D78151AA
:103A8000106E640E105C05E2200E92EC00F092ECD9
:103A900000F08151106E0A0E105C03E2200E92ECD1
:103AA00000F0800E016E815132EC00F0BA0E92EC03
:103AB00000F0BC0E92EC00F02F0E92EC00F0B40E71
:103AC00092EC00F012008251BB6FBC6BBBC014F0D3
:103AD000BCC015F00A0E186E196AE3EC02F0C16F53
:103AE000BBC014F0BCC015F00A0E186E196AE3ECE6
:103AF00002F01CC0C2F0550E92EC00F0610E92EC88
:103B000000F0BA0E92EC00F0200E92EC00F0800E65
:103B1000016E020E0B6EC15133EC00F02C0E92ECD4
:103B200000F0010E0B6EC25133EC00F012004FD8C2
:103B3000500E92EC00F0780E92EC00F092EC00F057
:103B4000200E92EC00F092EC00F0BC5306E1640E03
:103B5000BB5D03E2200E92EC00F0800E016E0B6A5A
:103B6000BBC01CF0BCC01DF035EC00F012002FD81B
:103B7000FE5306E0FE0E92EC00F0C00E92EC00F058
:103B8000010E446E060E445C08E2FE0E92EC00F05C
:103B9000140E92EC00F0442AF5E1BC5306E1640EE9
:103BA000BB5D03E2200E92EC00F0BC5306E10A0E6E
:103BB000BB5D03E2200E92EC00F0800E016E0B6AFA
:103BC000BBC01CF0BCC01DF035EC00F012006B0E49
:103BD000E75D010ED8A4000E316E080E49EC02F02C
:103BE000106E020E105CD8A4010E311604E0835151
:103BF000BB6FBC6B04D08351BC6F8451BB6F120090
:103C00006B0EE75D010ED8A4000E316E080E49EC74
:103C100002F0106E020E105CD8A4010E311604E002
:103C20008751BB6FBC6B03D08651BB6FBC6BBBC0F5
:103C300020F0BCC021F0880E186E130E196E3BECFC
:103C400003F0BB6F1DC0BCF0040E196E000ED2EC69
:103C500002F0BB6F15C0BCF0BBC014F0BCC015F0C7
:103C6000E80E186E030E196EE3EC02F0C16FBBC0D4
:103C700014F0BCC015F0E80E186E030E196EE3ECDC
:103C800002F01CC0BBF01DC0BCF0550E92EC00F061
:103C90004C0E92EC00F0200E92EC00F0800E016EC3
:103CA000C15132EC00F02C0E92EC00F0030E0B6EC2
:103CB000BBC01CF0BCC01DF035EC00F012006B0E58
:103CC000E75D010ED8A4000E316E080E49EC02F03B
:103CD000106E020E105CD8A4010E311604E089515A
:103CE000BB6FBC6B03D08751BB6FBC6BBBC014F008
:103CF000BCC015F00A0E186E196AE3EC02F0C16F31
:103D0000BBC014F0BCC015F00A0E186E196AE3ECC3
:103D100002F01CC0C2F0540E92EC00F0BD0E92EC0A
:103D200000F0BA0E92EC00F00A0EC15D03E2200E24
:103D300092EC00F0800E016EC15132EC00F02C0EBE
:103D400092EC00F0010E0B6EC25133EC00F0120049
:103D5000800E016E020E0B6E4A501DEC00F03A0E02
:103D600092EC00F0020E0B6E48501DEC00F01200B9
:103D7000EFDF3A0E92EC00F0800E016E020E0B6E39
:103D800046501DEC00F01200800E016E020E0B6E0C
:103D90004D501DEC00F02D0E92EC00F0020E0B6E5B
:103DA0004F501DEC00F01200EFDF2D0E92EC00F0F2
:103DB000800E016E020E0B6E51501DEC00F01200D1
:103DC00080EC21F0D2C017F0D1C016F0D0C015F0B1
:103DD000CFC014F01F6A1E6A030E1D6EE80E1C6E23
:103DE00074EC02F014C0BBF015C0BCF0D2C017F0E8
:103DF000D1C016F0D0C015F0CFC014F01F6A1E6AF3
:103E0000030E1D6EE80E1C6E74EC02F01CC0C3F0B5
:103E10001DC0C4F00A0EC15D03E2200E92EC00F05A
:103E2000800E016E0B6ABBC01CF0BCC01DF035ECEF
:103E300000F02C0E92EC00F0030E0B6EC3C01CF0D1
:103E4000C4C01DF035EC00F0A70E92EC00F0540E4B
:103E500092EC00F012009EEC21F03A0E49EC02F0D8
:103E6000D96F4AEC02F0DA6F4AEC02F0DB6F4AECF1
:103E700002F0DC6F38D94D0E92EC00F012009EEC8F
:103E800021F03A0E49EC02F0D96F4AEC02F0DA6FF9
:103E90004AEC02F0DB6F4AEC02F0DC6F0FD03FDA45
:103EA000610E49EC02F0D96F4AEC02F0DA6F4AEC8D
:103EB00002F0DB6F4AEC02F0DC6F00D0D951D55D27
:103EC000D96FDA51D659DA6FDB51D759DB6FDC5134
:103ED000D859DC6F9AEC23F0D2C017F0D1C016F09D
:103EE000D0C015F0CFC014F01F6A1E6A030E1D6EFD
:103EF000E80E1C6E74EC02F014C0BBF015C0BCF0F0
:103F0000D2C017F0D1C016F0D0C015F0CFC014F059
:103F10001F6A1E6A030E1D6EE80E1C6E74EC02F022
:103F20001FC0D2F01EC0D1F01DC0D0F01CC0CFF019
:103F3000BC5306E1640EBB5D03E2200E92EC00F080
:103F4000BC5306E10A0EBB5D03E2200E92EC00F0CA
:103F5000800E016E0B6ABBC01CF0BCC01DF035ECBE
:103F600000F02C0E92EC00F0030E0B6ED2C02AF083
:103F7000D1C029F0D0C028F0CFC027F063EC00F00A
:103F8000A70E92EC00F0DCC017F0DBC016F0DAC030
:103F900015F0D9C014F01F6A1E6A1D6A0A0E1C6E45
:103FA00074EC02F017C0DCF016C0DBF015C0DAF0DC
:103FB00014C0D9F0DCC017F0DBC016F0DAC015F081
:103FC000D9C014F01F6A1E6A1D6A0A0E1C6E74ECBA
:103FD00002F01CC0C2F0DCC017F0DBC016F0DAC083
:103FE00015F0D9C014F01F6A1E6A1D6A0A0E1C6EF5
:103FF00074EC02F017C0DCF016C0DBF015C0DAF08C
:1040000014C0D9F009EC3BF0D896DCBFD88609E49F
:10401000DC530AE1DB5108E1E80ED95D030EDA5901
:1040200003E2200E92EC00F0D896DCBFD88609E4BB
:10403000DC530AE1DB5308E1DA5306E1D9516308A6
:1040400003E3200E92EC00F0D896DCBFD88609E49A
:10405000DC530AE1DB5308E1DA5306E1D9510908E0
:1040600003E3200E92EC00F0800E016E0B6ADCC0C0
:104070002AF0DBC029F0DAC028F0D9C027F063ECC1
:1040800000F02C0E92EC00F0C25132EC00F04B0E1E
:1040900092EC00F04D0E92EC00F0BCEC39F0810E89
:1040A000056E800E0C6E256A2368246A010E266E4A
:1040B000565028EC02F0566ED8B0E0EF25F0EDD760
:1040C0002ED9610E49EC02F0D96F4AEC02F0DA6F9A
:1040D0004AEC02F0DB6F4AEC02F0DC6F04D8BC0E55
:1040E00092EC00F01200D951D55DD96FDA51D65952
:1040F000DA6FDB51D759DB6FDC51D859DC6FD896BA
:10410000DCBFD88638E4D951DA11DB11DC1133E099
:10411000D2C017F0D1C016F0D0C015F0CFC014F047
:104120001F6A1E6A030E1D6EE80E1C6EFAEC02F08A
:1041300017C02AF016C029F015C028F014C027F0C7
:104140002AC017F029C016F028C015F027C014F0B7
:10415000DCC01FF0DBC01EF0DAC01DF0D9C01CF0BF
:1041600074EC02F017C0D2F016C0D1F015C0D0F038
:1041700014C0CFF004D0D26BD16BD06BCF6BD2C058
:1041800017F0D1C016F0D0C015F0CFC014F01F6AE0
:104190001E6A1D6A0A0E1C6E74EC02F01FC013F03A
:1041A0001EC012F01DC011F01CC010F013BE0DD0C7
:1041B00011501210131003E1060E105C06E30A0EF4
:1041C000CF27000ED023D123D223D2C017F0D1C0E5
:1041D00016F0D0C015F0CFC014F01F6A1E6A1D6A19
:1041E0000A0E1C6E74EC02F017C0D2F016C0D1F0AB
:1041F00015C0D0F014C0CFF0D2C017F0D1C016F067
:10420000D0C015F0CFC014F01F6A1E6A1D6A0A0ED6
:104210001C6E74EC02F014C0BBF015C0BCF0D2C030
:1042200017F0D1C016F0D0C015F0CFC014F01F6A3F
:104230001E6A1D6A0A0E1C6E74EC02F01CC0C2F0ED
:10424000BBC014F0BCC015F0196A0A0E0BEC00F0EC
:10425000316EFEC014F0000E06EC00F0311603E0E3
:10426000200E92EC00F0800E016E0B6ABBC01CF0B9
:10427000BCC01DF035EC00F02C0E92EC00F0010EED
:104280000B6EC25133EC00F0010E92EC00F0020E06
:1042900092EC00F04B0E92EC00F0120031D8360E8A
:1042A000A96ECF514FEC02F0D0514FEC02F0D1513A
:1042B0004FEC02F0D2514FEC02F031D83E0EA96E15
:1042C000CF514FEC02F0D0514FEC02F0D1514FECF6
:1042D00002F0D2514FEC02F031D8420EA96ECF510C
:1042E0004FEC02F0D0514FEC02F0D1514FEC02F004
:1042F000D2514FEC02F0CD6BCE6BD36BD46B12006E
:10430000360E49EC02F0CF6F4AEC02F0D06F4AEC67
:1043100002F0D16F4AEC02F0D26F1FD812003E0EAD
:1043200049EC02F0CF6F4AEC02F0D06F4AEC02F099
:10433000D16F4AEC02F0D26F10D81200420E49EC55
:1043400002F0CF6F4AEC02F0D06F4AEC02F0D16F6E
:104350004AEC02F0D26F01D81200D351CF27D451CA
:10436000D023000ED123D2231200320E49EC02F0EA
:10437000D96F4AEC02F0DA6F4AEC02F0DB6F4AECDC
:1043800002F0DC6FD951D55D276EDA51D659286E0F
:10439000DB51D759296EDC51D8592A6E2AC017F043
:1043A00029C016F028C015F027C014F01F6A0F0EA0
:1043B0001E6E420E1D6E400E1C6E74EC02F01FC08D
:1043C000DCF01EC0DBF01DC0DAF01CC0D9F0D896BE
:1043D000DCBFD88609E49F0ED95D860EDA59010E3E
:1043E000DB59000EDC593FE2DCC017F0DBC016F0F1
:1043F000DAC015F0D9C014F01F6A1E6A1D6A640E77
:104400001C6E74EC02F01CC0C2F0DCC017F0DBC004
:1044100016F0DAC015F0D9C014F01F6A1E6A1D6AC2
:10442000640E1C6E74EC02F017C0DCF016C0DBF0FA
:1044300015C0DAF014C0D9F0800E016E030E0B6EB9
:10444000DCC02AF0DBC029F0DAC028F0D9C027F0A0
:1044500063EC00F02E0E92EC00F0020E0B6EC251D7
:1044600033EC00F044D0DCC017F0DBC016F0DAC04B
:1044700015F0D9C014F01F6A1E6A1D6A640E1C6E06
:1044800074EC02F01CC0C2F0C2C014F00A0EE0ECE2
:1044900002F0C26FDCC017F0DBC016F0DAC015F016
:1044A000D9C014F01F6A1E6A1D6A640E1C6E74EC7B
:1044B00002F017C0DCF016C0DBF015C0DAF014C053
:1044C000D9F0800E016E040E0B6EDCC02AF0DBC04A
:1044D00029F0DAC028F0D9C027F063EC00F02E0EE6
:1044E00092EC00F0010E0B6EC25133EC00F0BA0EEC
:1044F00092EC00F0BC0E92EC00F01200550E49EC6C
:1045000002F0D96F4AEC02F0DA6F4AEC02F0DB6F8E
:104510004AEC02F0DC6F29D04A0E49EC02F04D6EF5
:104520004B0E49EC02F04F6E4C0E49EC02F0516E0E
:1045300012004D0E49EC02F0D96F4AEC02F0DA6F2E
:104540004AEC02F0DB6F4AEC02F0DC6F0ED0510E49
:1045500049EC02F0D96F4AEC02F0DA6F4AEC02F053
:10456000DB6F4AEC02F0DC6F00D0D951D55DD96F1A
:10457000DA51D659DA6FDB51D759DB6FDC51D85994
:10458000DC6FDCC017F0DBC016F0DAC015F0D9C064
:1045900014F01F6A1E6A1D6A640E1C6E74EC02F031
:1045A00017C0DCF016C0DBF015C0DAF014C0D9F08B
:1045B000070EF76E3E0EF66E8AEC00F01200010E4A
:1045C000C95DD8B419EC18F0020EC95DD8B42BEC53
:1045D0001FF0030EC95DD8B4E0EC1EF0040EC95DF7
:1045E000D8B460EC20F0050EC95DD8B490EC19F099
:1045F000060EC95DD8B4C3EC19F0070EC95DD8B476
:1046000033EC1AF0080EC95DD8B4A5EC1AF0090E07
:10461000C95DD8B45FEC1EF00A0EC95DD8B4E1ECF8
:104620001AF00B0EC95DD8B401EC1BF00C0EC95D7D
:10463000D8B411EC1BF00D0EC95DD8B48BEC1BF097
:104640000E0EC95DD8B400EC1CF00F0EC95DD8B4D5
:104650003FEC1DF0100EC95DD8B463EC1DF0110ED7
:10466000C95DD8B400EC1EF0120EC95DD8B497EC49
:104670001DF0130EC95DD8B4A8EC1EF0140EC95D70
:10468000D8B4B8EC1EF0150EC95DD8B4C4EC1EF059
:10469000160EC95DD8B4D4EC1EF0170EC95DD8B49F
:1046A00064DE180EC95DD8B422EC39F0190EC95D6C
:1046B000D8B470EC1AF01A0EC95D06E1070EF76E59
:1046C000480EF66E8AEC00F01B0EC95D18E3480E2A
:1046D00092EC00F0650E92EC00F0200E92EC00F0EF
:1046E000B30E92EC00F0B80E92EC00F0B70E92EC24
:1046F00000F0BD0E92EC00F02E0E92EC00F01200D5
:10470000446A2F0E445C08E2F36A00EE5AF044500B
:10471000F3CFEBFF442AF5E11200446A2F0E445C0C
:1047200008E2F36A00EE8AF04450F3CFEBFF442A2C
:10473000F5E11200FE0E92EC00F0010E92EC00F09A
:1047400002EC3BF012005D50106E700E105C18E130
:1047500009EC3BF0D90E92EC00F02D0E92EC00F03B
:10476000800E016E0B6ABBC01CF0BCC01DF035ECA6
:1047700000F02B0E92EC00F0DA0E92EC00F001D07B
:1047800055861200D7DF450E92EC00F0BA0E92EC7F
:1047900000F0700E92EC00F0610E92EC00F0BD0E95
:1047A00092EC00F0200E92EC00F0800E016E020EF2
:1047B0000B6E45281C6E1D6A1D3635EC00F009ECA9
:1047C0003BF0C00EE75D1AE1080E49EC02F0106EF6
:1047D000105206E1070EF76E520EF66E8AEC00F0EC
:1047E000080E49EC02F0106E010E105C06E1070E97
:1047F000F76E5A0EF66E8AEC00F022D06B0EE75D73
:104800001AE1080E49EC02F0106E105206E1070E94
:10481000F76E620EF66E8AEC00F0080E49EC02F0BC
:10482000106E020E105C06E1070EF76E6A0EF66E51
:104830008AEC00F005D0800E016EE7511CEC00F010
:104840001200FB6B558655A64BD1559673DFFB5373
:104850005AE181BC27D0FE0E92EC00F0280E92ECBB
:1048600000F0FE0E92EC00F0080E92EC00F0FE0E4E
:1048700092EC00F0010E92EC00F0FE0E92EC00F0D3
:10488000060E92EC00F0FE0E92EC00F00C0E92EC94
:1048900000F0020E196E260E5DEC02F060EC33F0B3
:1048A00038EF05F0D90E92EC00F0480E92EC00F0D3
:1048B000610E92EC00F0BB0E92EC00F0200E92EC38
:1048C00000F02D0E92EC00F092EC00F03E0E92EC17
:1048D00000F009EC3BF0DA0E92EC00F04D0E92EC99
:1048E00000F0650E92EC00F0BD0E92EC00F0200E90
:1048F00092EC00F0A40E92EC00F0BA0E92EC00F0F4
:10490000700E92EC00F0010EFB5D32E1A70E92EC0E
:1049100000F0690E92EC00F0C00E92EC00F0B80EC0
:1049200092EC00F0BB0E92EC00F0C40E92EC00F0A2
:10493000BD0E92EC00F02E0E92EC00F009EC3BF074
:10494000790E92EC00F0BE0E92EC00F0700E92EC3C
:1049500000F0610E92EC00F0B30E92EC00F02E0E1F
:1049600092EC00F0200E92EC00F0030E92EC00F0BE
:10497000020EFB5D32E1E00E92EC00F0690E92EC6B
:1049800000F0610E92EC00F0B40E92EC00F0BD0E5F
:1049900092EC00F06F0E92EC00F0630E92EC00F0DF
:1049A000BF0E92EC00F009EC3BF0690E92EC00F0C7
:1049B000BD0E92EC00F0B60E92EC00F0650E92EC9B
:1049C00000F0BA0E92EC00F0BF0E92EC00F02E0E4A
:1049D00092EC00F0030E92EC00F0030EFB5D32E16E
:1049E0004B0E92EC00F0650E92EC00F0700E92EC23
:1049F00000F0790E92EC00F0B30E92EC00F0610E34
:104A000092EC00F0BD0E92EC00F02E0E92EC00F055
:104A100009EC3BF0690E92EC00F0BD0E92EC00F058
:104A2000B60E92EC00F0650E92EC00F0BA0E92EC2D
:104A300000F0BF0E92EC00F02E0E92EC00F0050E8E
:104A400092EC00F0040EFB5D32E1A90E92EC00F056
:104A5000630E92EC00F0BF0E92EC00F0610E92EC4F
:104A600000F0BD0E92EC00F06F0E92EC00F0B30E71
:104A700092EC00F02E0E92EC00F009EC3BF0A00E50
:104A800092EC00F04B0E92EC00F0200E92EC00F055
:104A9000200E92EC00F0200E92EC00F0200E92EC32
:104AA00000F0200E92EC00F0050E92EC00F0050EE6
:104AB000FB5D16E1420E92EC00F0650E92EC00F008
:104AC000700E92EC00F0630E92EC00F0690E92EC26
:104AD00000F0C70E92EC00F009EC3BF0F0EC39F07E
:104AE000BCEC39F0810E056E800E0C6E256A2368D1
:104AF000246A010E266E565028EC02F0566E39E2FA
:104B0000810E056E400E0C6E256A2368246A010E24
:104B1000266E575028EC02F0576E3FE2810E056E6C
:104B2000200E0C6E256A2368246A010E266E5850EA
:104B300028EC02F0586E0FE2810E056E100E0C6E1E
:104B4000256A2368246A010E266E595028EC02F06B
:104B5000596E09E278D65586FB5303E195EF09F0CB
:104B600001D0FB0770D65586050EFB5DD8A0FB2B48
:104B70006AD6558681BC0AD0558A030EFB5DD8B42F
:104B8000CFEF2CF0040EFB5DD8B452D2FB5302E001
:104B9000FB6B02D004EF05F056D6FB5307E1A96A80
:104BA00045504FEC02F004EF05F008D0010EFB5D1C
:104BB00006E0020EFB5DD8B4E0EF2AF044D6FC6BB1
:104BC0005588FE6B55A8F1D15598B4DDFC533AE1F8
:104BD00055B20DEC17F0A80E92EC00F0700E92ECAE
:104BE00000F06F0E92EC00F0B20E92EC00F0690E45
:104BF00092EC00F0B40E92EC00F04B0E92EC00F050
:104C00004D0E92EC00F009EC3BF0800E016E080EA8
:104C10000B6ED8C017F0D7C016F0D6C015F0D5C0AF
:104C200014F01F6A1E6A1D6A640E1C6E74EC02F09A
:104C300017C02AF016C029F015C028F014C027F0BC
:104C400063EC00F0010EFC5D1FE155B20DEC17F0B6
:104C50004F0E92EC00F0E30E92EC00F06F0E92EC2F
:104C600000F0BC0E92EC00F0650E92EC00F0BF0E6E
:104C700092EC00F0700E92EC00F0030E92EC00F05B
:104C800009EC3BF0B5EC21F0020EFC5D1CE1510E8D
:104C900092EC00F02E0E92EC00F0B70E92EC00F0C9
:104CA000610E92EC00F0B40E92EC00F02E0E92EC3D
:104CB00000F0200E92EC00F0030E92EC00F009ECF4
:104CC0003BF0E0EC1EF0030EFC5D1CE1510E92EC9B
:104CD00000F02E0E92EC00F0BE0E92EC00F06F0E83
:104CE00092EC00F0040E92EC00F0B70E92EC00F0A3
:104CF000E30E92EC00F0030E92EC00F009EC3BF0B6
:104D000060EC20F0040EFC5D1CE1510E92EC00F012
:104D10002E0E92EC00F0630E92EC00F0650E92EC19
:104D200000F0700E92EC00F0E30E92EC00F0BD0E7D
:104D300092EC00F0030E92EC00F009EC3BF02BEC4F
:104D40001FF0050EFC5D20E14D0E92EC00F0610EAF
:104D500092EC00F0630E92EC00F0BB0E92EC00F0CF
:104D60006F0E92EC00F04B0E92EC00F0BC0E92EC49
:104D700000F0030E92EC00F009EC3BF0070EF76E2A
:104D8000720EF66E8AEC00F0060EFC5D20E14D0E10
:104D900092EC00F0610E92EC00F0630E92EC00F0E9
:104DA000BB0E92EC00F06F0E92EC00F0E00E92EC75
:104DB00000F0BF0E92EC00F0030E92EC00F009EC54
:104DC0003BF0070EF76E7C0EF66E8AEC00F0070ED5
:104DD000FC5D20E1500E92EC00F0650E92EC00F0CC
:104DE000BC0E92EC00F02E0E92EC00F0A10E92ECB4
:104DF00000F0500E92EC00F04D0E92EC00F0030E1D
:104E000092EC00F009EC3BF0070EF76E860EF66EA2
:104E10008AEC00F0080EFC5D20E1430E92EC00F0FD
:104E2000B30E92EC00F0690E92EC00F0C00E92EC22
:104E300000F0BA0E92EC00F0B80E92EC00F0200EEA
:104E400092EC00F0030E92EC00F009EC3BF0070E40
:104E5000F76E900EF66E8AEC00F0090EFC5D20E114
:104E6000E00E92EC00F0650E92EC00F0BF0E92ECBA
:104E700000F0BD0E92EC00F02E0E92EC00F0430E0E
:104E800092EC00F0650E92EC00F0BA0E92EC00F09D
:104E900009EC3BF0070EF76E9A0EF66E8AEC00F006
:104EA0000A0EFC5D20E1A80E92EC00F0700E92EC70
:104EB00000F06F0E92EC00F0BE0E92EC00F02E0EA1
:104EC00092EC00F0430E92EC00F0650E92EC00F0D4
:104ED000BA0E92EC00F009EC3BF0070EF76EA40E50
:104EE000F66E8AEC00F00B0EFC5D20E14D0E92ECAC
:104EF00000F0610E92EC00F0780E92EC00F0AC0E37
:104F000092EC00F0B30E92EC00F0B80E92EC00F0D0
:104F1000E30E92EC00F0030E92EC00F009EC3BF093
:104F2000070EF76EAE0EF66E8AEC00F00C0EFC5D0E
:104F30003CE13F6A43BE19D040504110421043103B
:104F400014E03EC017F03DC016F03CC015F03BC069
:104F500014F043C01FF042C01EF041C01DF040C01D
:104F60001CF074EC02F014C03FF0430E92EC00F021
:104F7000650E92EC00F0700E92EC00F0AC0E92EC2C
:104F800000F0B30E92EC00F0B80E92EC00F0E30EDD
:104F900092EC00F0030E92EC00F009EC3BF0070EEF
:104FA000F76EB80EF66E8AEC00F0BCEC39F0810EAC
:104FB000056E800E0C6E256A2368246A010E266E2B
:104FC000565028EC02F0566ED8B06CEF2FF0810EE0
:104FD000056E400E0C6E256A2368246A010E266E4B
:104FE000575028EC02F0576ED8B06FEF2FF0810EBB
:104FF000056E200E0C6E256A2368246A010E266E4B
:10500000585028EC02F0586ED8B02FEF2FF0810ED8
:10501000056E100E0C6E256A2368246A010E266E3A
:10502000595028EC02F0596ED8B047EF2FF0CAD58E
:10503000FC6B558681BC559A55A64BD255969AEC79
:1050400023F0FC532CE1A10E92EC00F06F0E92ECD9
:1050500000F0E30E92EC00F0B80E92EC00F0BD0E02
:1050600092EC00F0610E92EC00F009EC3BF0BD0E0A
:1050700092EC00F0610E92EC00F0630E92EC00F006
:10508000BF0E92EC00F0700E92EC00F02E0E92EC3F
:1050900000F0200E92EC00F0030E92EC00F0010EF6
:1050A000FC5D32E1A80E92EC00F0700E92EC00F084
:1050B0006F0E92EC00F0E30E92EC00F0790E92ECA1
:1050C00000F0BA0E92EC00F0BF0E92EC00F02E0E43
:1050D00092EC00F009EC3BF0E40E92EC00F06F0E65
:1050E00092EC00F0700E92EC00F0630E92EC00F087
:1050F0002E0E92EC00F0200E92EC00F0200E92ECBE
:1051000000F0030E92EC00F0020EFC5D4CE1420E4A
:1051100092EC00F0BE0E92EC00F0700E92EC00F0FB
:10512000B80E92EC00F0630E92EC00F0BA0E92EC26
:1051300000F009EC3BF0030E49EC02F0106E010E9A
:10514000105C19E1AA0E92EC00F0610E92EC00F0F6
:10515000B70E92EC00F06F0E92EC00F0B30E92ECF2
:1051600000F02E0E92EC00F0200E92EC00F03E0EBD
:1051700092EC00F018D0480E92EC00F0650E92EC24
:1051800000F0AA0E92EC00F0610E92EC00F0B70E67
:1051900092EC00F06F0E92EC00F0B30E92EC00F087
:1051A0003E0E92EC00F0030EFC5D21E1A70E92ECA6
:1051B00000F06F0E92EC00F0B40E92EC00F06F0E67
:1051C00092EC00F0BF0E92EC00F0B80E92EC00F002
:1051D000BE0E92EC00F009EC3BF0040E49EC02F03C
:1051E000106E010E105C02E1D2D901D0B7D9040EC5
:1051F000FC5D2FE1540E92EC00F0700E92EC00F08A
:10520000B80E92EC00F0B30E92EC00F0610E92EC4E
:1052100000F0BB0E92EC00F02E0E92EC00F009ECC8
:105220003BF0630E92EC00F0BD0E92EC00F0790EB4
:1052300092EC00F0200E92EC00F0200E92EC00F0C8
:10524000200E92EC00F0200E92EC00F0030E92EC97
:1052500000F0050EFC5D3AE1AB0E92EC00F0610E41
:1052600092EC00F0630E92EC00F0BF0E92EC00F0B6
:105270006F0E92EC00F0BF0E92EC00F0610E92EC1B
:1052800000F009EC3BF0050E49EC02F0106E010E47
:10529000105C04E1320E92EC00F003D0310E92EC7F
:1052A00000F0200E92EC00F0A10E92EC00F0E50E62
:1052B00092EC00F0200E92EC00F0200E92EC00F048
:1052C000200E92EC00F03E0E92EC00F0060EFC5D1B
:1052D000D8A45ED0AB0E92EC00F0610E92EC00F020
:1052E000630E92EC00F02B0E92EC00F0540E92EC58
:1052F00000F0650E92EC00F0BC0E92EC00F0BE0ED9
:1053000092EC00F009EC3BF0060E49EC02F0106E56
:1053100010520CE1AB0E92EC00F0610E92EC00F03A
:10532000630E92EC00F0200E92EC00F0060E49ECB9
:1053300002F0106E010E105C0CE1540E92EC00F0C5
:10534000610E92EC00F0BA0E92EC00F0200E92EC9E
:1053500000F0060E49EC02F0106E020E105C0CE13B
:10536000540E92EC00F0650E92EC00F0BC0E92EC44
:1053700000F0BE0E92EC00F0200E92EC00F0200E39
:1053800092EC00F0200E92EC00F03E0E92EC00F059
:10539000070EFC5D24E1A80E92EC00F06F0E92EC7B
:1053A00000F0B30E92EC00F0690E92EC00F0E30E08
:1053B00092EC00F06F0E92EC00F0BC0E92EC00F05C
:1053C0002E0E92EC00F009EC3BF0070E49EC02F0D7
:1053D000106E010E105C02E1DAD801D0BFD8080EC1
:1053E000FC5DD8A476D04D0E92EC00F0490E92EC04
:1053F00000F04B0E92EC00F0410E92EC00F0430EE8
:1054000092EC00F0200E92EC00F0200E92EC00F0F6
:105410003E0E92EC00F009EC3BF0080E49EC02F075
:10542000106E105218E1370E92EC00F02E0E92EC36
:1054300000F0360E92EC00F02D0E92EC00F0310EE2
:1054400092EC00F0300E92EC00F02E0E92EC00F098
:10545000330E92EC00F0080E49EC02F0106E010ED3
:10546000105C18E1200E92EC00F0310E92EC00F08E
:10547000300E92EC00F02E0E92EC00F0330E92EC17
:1054800000F02B0E92EC00F0200E92EC00F0200EBB
:1054900092EC00F0080E49EC02F0106E020E105C67
:1054A00018E1200E92EC00F0200E92EC00F0310E8C
:1054B00092EC00F0310E92EC00F02E0E92EC00F027
:1054C000340E92EC00F0200E92EC00F0200E92ECE4
:1054D00000F0BCEC39F0810E056E800E0C6E256A72
:1054E0002368246A010E266E565028EC02F0566E90
:1054F000D8B06CEF2FF055BA10D0810E056E400E6B
:105500000C6E256A2368246A010E266E575028EC1B
:1055100002F0576ED8B06FEF2FF0810E056E200E9F
:105520000C6E256A2368246A010E266E585028ECFA
:1055300002F0586ED8B02FEF2FF0810E056E100ECE
:105540000C6E256A2368246A010E266E595028ECD9
:1055500002F0596ED8B047EF2FF06CD5BE0E92EC2A
:1055600000F06F0E92EC00F0BA0E92EC00F0610EBB
:1055700092EC00F0B70E92EC00F02E0E92EC00F0E0
:10558000200E92EC00F03E0E92EC00F01200BD0EE8
:1055900092EC00F0650E92EC00F0BE0E92EC00F082
:1055A0006F0E92EC00F0BA0E92EC00F0610E92ECED
:1055B00000F0B70E92EC00F03E0E92EC00F01200FC
:1055C000FC6B558655A6AAD155969AEC23F0FE6B36
:1055D000FC532FE1A80E92EC00F06F0E92EC00F05D
:1055E000BC0E92EC00F0B80E92EC00F0BB0E92EC08
:1055F00000F0BA0E92EC00F0B80E92EC00F009EC5C
:105600003BF0450E92EC00F0430E92EC00F0A90E38
:1056100092EC00F0E00E92EC00F0200E92EC00F024
:10562000200E92EC00F0200E92EC00F0030E92ECB3
:1056300000F0010EFC5D2FE1A80E92EC00F06F0E61
:1056400092EC00F0BC0E92EC00F0B80E92EC00F080
:10565000BB0E92EC00F0BA0E92EC00F0B80E92EC99
:1056600000F009EC3BF06F0E92EC00F0C00E92ECF3
:1056700000F0B80E92EC00F0630E92EC00F0BF0E5A
:1056800092EC00F02E0E92EC00F0200E92EC00F066
:105690003E0E92EC00F0020EFC5D2FE1A80E92ECA3
:1056A00000F06F0E92EC00F0BC0E92EC00F0B80E21
:1056B00092EC00F0BB0E92EC00F0BA0E92EC00F00F
:1056C000B80E92EC00F009EC3BF0A80E92EC00F062
:1056D0006F0E92EC00F0BF0E92EC00F06F0E92ECA9
:1056E00000F0C00E92EC00F0BD0E92EC00F02E0E19
:1056F00092EC00F0030E92EC00F0030EFC5D32E140
:10570000A80E92EC00F06F0E92EC00F0BC0E92EC42
:1057100000F02E0E92EC00F0A80E92EC00F06F0E4E
:1057200092EC00F0BF0E92EC00F02E0E92EC00F026
:1057300009EC3BF06F0E92EC00F0C00E92EC00F022
:10574000B80E92EC00F0630E92EC00F0BF0E92ECFB
:1057500000F02E0E92EC00F0200E92EC00F03E0EC7
:1057600092EC00F0040EFC5D2FE1E00E92EC00F0F4
:10577000610E92EC00F0BF0E92EC00F0C00E92ECC5
:1057800000F0B80E92EC00F0BA0E92EC00F0B80EF9
:1057900092EC00F009EC3BF0410E92EC00F0E10ECF
:1057A00092EC00F0A80E92EC00F0200E92EC00F0CB
:1057B000200E92EC00F0200E92EC00F0200E92EC05
:1057C00000F0030E92EC00F0050EFC5D32E14B0E92
:1057D00092EC00F06F0E92EC00F0BC0E92EC00F038
:1057E000BE0E92EC00F0BB0E92EC00F0650E92EC57
:1057F00000F0BA0E92EC00F02D0E92EC00F009ECE5
:105800003BF0BF0E92EC00F0610E92EC00F0E50E62
:1058100092EC00F0690E92EC00F0C70E92EC00F0F2
:10582000200E92EC00F0200E92EC00F0030E92ECB1
:1058300000F0060EFC5D2FE1A80E92EC00F0610E68
:1058400092EC00F0630E92EC00F0BE0E92EC00F0D1
:105850006F0E92EC00F0700E92EC00F0BF0E92EC26
:1058600000F009EC3BF0450E92EC00F0A00E92EC3B
:1058700000F04B0E92EC00F0200E92EC00F0200EA7
:1058800092EC00F0200E92EC00F0200E92EC00F072
:10589000030E92EC00F0070EFC5D1EE16CEC11F0C3
:1058A000A5EC1AF002EC3BF0B7EC1DF009EC3BF074
:1058B00033EC1AF009EC3BF0010E446E060E445C2A
:1058C00008E2FE0E92EC00F0140E92EC00F0442A76
:1058D000F5E1E1EC1AF05586080EFC5D1FE1EDECF8
:1058E00011F002EC3BF0A80E92EC00F0700E92EC7E
:1058F00000F06F0E92EC00F0BE0E92EC00F0790E0C
:1059000092EC00F0630E92EC00F0BA0E92EC00F014
:10591000B80E92EC00F009EC3BF05586BCEC39F087
:10592000810E056E800E0C6E256A2368246A010EB6
:10593000266E565028EC02F0566ED8B06CEF2FF061
:10594000810E056E400E0C6E256A2368246A010ED6
:10595000266E575028EC02F0576ED8B06FEF2FF03C
:10596000810E056E200E0C6E256A2368246A010ED6
:10597000266E585028EC02F0586ED8B070D2810EC6
:10598000056E100E0C6E256A2368246A010E266EC1
:10599000595028EC02F0596ED8B079D213D6FC6B6E
:1059A000558681BC559A55A602D255969AEC23F09D
:1059B000FC5332E14B0E92EC00F0610E92EC00F0E1
:1059C000BB0E92EC00F0690E92EC00F0B20E92EC7D
:1059D00000F0700E92EC00F0790E92EC00F0B30E35
:1059E00092EC00F009EC3BF0E30E92EC00F0700E4C
:1059F00092EC00F06F0E92EC00F0630E92EC00F06F
:105A0000650E92EC00F0BB0E92EC00F0C40E92EC2E
:105A100000F0030E92EC00F0010EFC5D2CE14F0E45
:105A200092EC00F0B20E92EC00F0650E92EC00F0F9
:105A3000700E92EC00F0BF0E92EC00F0B80E92ECFB
:105A400000F009EC3BF0580E92EC00F0580E92EC8E
:105A500000F0200E92EC00F0200E92EC00F0200EF0
:105A600092EC00F0200E92EC00F0200E92EC00F090
:105A7000030E92EC00F0020EFC5D32E1A90E92ECF6
:105A800000F0630E92EC00F0BF0E92EC00F0610E9D
:105A900092EC00F0BD0E92EC00F06F0E92EC00F074
:105AA000B30E92EC00F02E0E92EC00F009EC3BF0FD
:105AB000470E92EC00F0300E92EC00F0580E92EC93
:105AC00000F0580E92EC00F0200E92EC00F0200E48
:105AD00092EC00F0200E92EC00F0030E92EC00F03D
:105AE000030EFC5D32E1A90E92EC00F0630E92EC25
:105AF00000F0BF0E92EC00F0610E92EC00F0BD0ED3
:105B000092EC00F06F0E92EC00F0B30E92EC00F00D
:105B10002E0E92EC00F009EC3BF0470E92EC00F0F8
:105B2000300E92EC00F0420E92EC00F0200E92EC5F
:105B300000F0200E92EC00F0200E92EC00F0200E0F
:105B400092EC00F0030E92EC00F0040EFC5D1BE101
:105B5000A00E92EC00F0650E92EC00F0BD0E92ECFF
:105B600000F0B70E92EC00F06F0E92EC00F0BD0E5C
:105B700092EC00F0610E92EC00F0630E92EC00F0FB
:105B800009EC3BF053D9050EFC5D18E1420E92EC96
:105B900000F0650E92EC00F0BD0E92EC00F0BF0E2E
:105BA00092EC00F0B80E92EC00F0BB0E92EC00F01C
:105BB0002E0E92EC00F009EC3BF038D9060EFC5D9D
:105BC0001BE1430E92EC00F0680E92EC00F0650EC3
:105BD00092EC00F0630E92EC00F06B0E92EC00F091
:105BE000450E92EC00F06E0E92EC00F0670E92EC17
:105BF00000F009EC3BF01AD9070EFC5D32E1A80E6B
:105C000092EC00F0690E92EC00F0E30E92EC00F0E2
:105C1000690E92EC00F0B40E92EC00F0700E92EC73
:105C200000F0690E92EC00F0B30E92EC00F009EC7B
:105C30003BF0E30E92EC00F0700E92EC00F06F0E71
:105C400092EC00F0630E92EC00F0650E92EC00F026
:105C5000BB0E92EC00F0C70E92EC00F0030E92EC3B
:105C600000F0080EFC5D32E14B0E92EC00F0650E88
:105C700092EC00F0700E92EC00F0790E92EC00F0D5
:105C8000B30E92EC00F0610E92EC00F0BD0E92ECBF
:105C900000F02E0E92EC00F009EC3BF0500E92EC6E
:105CA00000F0580E92EC00F0580E92EC00F0200E2E
:105CB00092EC00F0200E92EC00F0200E92EC00F03E
:105CC000200E92EC00F0030E92EC00F0090EFC5D49
:105CD0001BE1410E92EC00F0E30E92EC00F0630E3B
:105CE00092EC00F06F0E92EC00F0700E92EC00F06F
:105CF000B20E92EC00F0650E92EC00F0700E92EC99
:105D000000F009EC3BF092D80A0EFC5D1BE14B0E53
:105D100092EC00F0790E92EC00F0BF0E92EC00F0E5
:105D2000A40E92EC00F0610E92EC00F0BE0E92EC2C
:105D300000F0610E92EC00F0BB0E92EC00F009EC6A
:105D40003BF074D80B0EFC5D32E14F0E92EC00F08C
:105D5000C00E92EC00F0B80E92EC00F0630E92ECE4
:105D600000F0BF0E92EC00F0540E92EC00F0610EC9
:105D700092EC00F0B20E92EC00F009EC3BF0610EF8
:105D800092EC00F0E30E92EC00F0610E92EC00F069
:105D9000BE0E92EC00F0BF0E92EC00F02E0E92ECD4
:105DA00000F0200E92EC00F03E0E92EC00F0BCEC05
:105DB00039F0810E056E800E0C6E256A2368246A08
:105DC000010E266E565028EC02F0566ED8B084D0E4
:105DD00055BA0FD0810E056E400E0C6E256A2368F1
:105DE000246A010E266E575028EC02F0576ED8B088
:105DF00076D0810E056E200E0C6E256A2368246A0B
:105E0000010E266E585028EC02F0586E28E2810EE2
:105E1000056E100E0C6E256A2368246A010E266E2C
:105E2000595028EC02F0596E32E2BBD5BA0E92EC12
:105E300000F0650E92EC00F0700E92EC00F0790E1E
:105E400092EC00F0B30E92EC00F02E0E92EC00F00B
:105E5000200E92EC00F0030E92EC00F01200FC53C6
:105E6000D8A4FC07010EFB5DD8B4E0EF25F0020ECC
:105E7000FB5DD8B4E1EF2AF0030EFB5DD8B490D5FA
:105E8000040EFB5DD8B419EF28F023EF24F0010EC7
:105E9000FB5D06E10C0EFC5DD8A0FC2BE0EF25F0CD
:105EA000020EFB5D06E1070EFC5DD8A0FC2BE1EFC6
:105EB0002AF0030EFB5D05E10B0EFC5DD8A0FC2B68
:105EC0006FD5040EFB5D06E1080EFC5DD8A0FC2B2F
:105ED00019EF28F023EF24F0558623EF24F05586A0
:105EE000010EFB5D16E1010EFC53D8A4000E316ECD
:105EF000090EFC5D010ED8A4000E31120A0EFC5DE5
:105F0000010ED8A4000E311203E0E2EF25F001D01B
:105F100016D2020EFB5D22E1FC53D8B422EF0DF045
:105F2000010EFC5DD8B4B3EF12F0020EFC5DD8B4E4
:105F3000E9EF0DF0030EFC5DD8B4EDEF12F0040EA6
:105F4000FC5DD8B4A6EF35F0050EFC5DD8B44DEF7E
:105F50000FF0060EFC5DD8B413EF37F0030EFB5DB7
:105F6000D8A450D0FC530CE16F50BC6F7050BB6F85
:105F7000BC51BB1103E1C5EF15F002D0CFEF2CF0FF
:105F8000010EFC5DD8B4A9EF13F0020EFC5DD8B48D
:105F9000A9EF13F0030EFC5DD8B4A9EF13F0040EC3
:105FA000FC5DD8B4B6EF34F0050EFC5DD8B4B6EFA6
:105FB00034F0060EFC5DD8B4B6EF34F0070EFC5D8D
:105FC000D8B4B6EF34F0080EFC5DD8B4A9EF13F0E6
:105FD000090EFC5DD8B4A9EF13F00A0EFC5DD8B42D
:105FE000A9EF13F00B0EFC5D0DE1070EF76EC20E6C
:105FF000F66E8AEC00F0030E196EE80E5DEC02F00E
:1060000002EF05F0040EFB5DD8A484D0FC5304E13C
:10601000FEEC06F0AAEF07F0010EFC5DD8B47CD0D0
:10602000020EFC5DD8B46FD1030EFC5DD8B479D1FB
:10603000040EFC5DD8B4E8D0050EFC5D14E1050E3D
:1060400049EC02F0106E010E105C06E1050EA96E1F
:10605000000E4FEC02F005D0050EA96E010E4FECBC
:1060600002F019EF28F0060EFC5D29E1060E49EC5E
:1060700002F0106E105207E1060EA96E010E4FECF1
:1060800002F019EF28F0060E49EC02F0106E010E36
:10609000105C07E1060EA96E020E4FEC02F019EF3C
:1060A00028F0060E49EC02F0106E020E105C07E1BB
:1060B000060EA96E000E4FEC02F019EF28F0070E45
:1060C000FC5D14E1070E49EC02F0106E010E105C4D
:1060D00006E1070EA96E000E4FEC02F005D0070E88
:1060E000A96E010E4FEC02F019EF28F0080EFC5DCE
:1060F00011E1080E49EC02F0106E1028B96F030E82
:10610000B95DD8B0B96B080EA96EB9514FEC02F069
:1061100019EF28F023EF24F0558655A636D0559672
:106120009AEC23F0020E49EC02F0B96F510E92EC9A
:1061300000F0200E92EC00F0E40E92EC00F06F0EF6
:1061400092EC00F0700E92EC00F0630E92EC00F016
:106150002E0E92EC00F0D90E92EC00F009EC3BF020
:10616000B5D8800E016EB95132EC00F0BC0E92EC45
:1061700000F0BB0E92EC00F02F0E92EC00F0780EC7
:1061800092EC00F0DA0E92EC00F0BCEC39F0810EEB
:10619000056E800E0C6E256A2368246A010E266E39
:1061A000565028EC02F0566ED8B019EF28F0810E48
:1061B000056E200E0C6E256A2368246A010E266E79
:1061C000585028EC02F0586E0FE2810E056E100E4A
:1061D0000C6E256A2368246A010E266E595028EC3D
:1061E00002F0596E09E299D75586B92B020EA96EB5
:1061F000B9514FEC02F091D75586B907020EA96E3E
:10620000B9514FEC02F089D7558655A630D0559636
:106210009AEC23F0010E49EC02F0B96F430E92ECB8
:1062200000F06F0E92EC00F0BD0E92EC00F0200E2C
:1062300092EC00F0580E92EC00F0B30E92EC00F0ED
:106240002E0E92EC00F009EC3BF0D90E92EC00F02F
:106250002B0E92EC00F03AD8800E016EB95132EC60
:1062600000F02D0E92EC00F0DA0E92EC00F0BCEC97
:1062700039F0810E056E800E0C6E256A2368246A43
:10628000010E266E565028EC02F0566ED8B019EF6B
:1062900028F0810E056E200E0C6E256A2368246A94
:1062A000010E266E585028EC02F0586E1CE2810E4A
:1062B000056E100E0C6E256A2368246A010E266E88
:1062C000595028EC02F0596E16E29FD7640EB95D62
:1062D00003E2200E92EC00F00A0EB95D03E2200EFC
:1062E00092EC00F012005586B92B010EA96EB9513F
:1062F0004FEC02F08AD75586B907010EA96EB95145
:106300004FEC02F082D7010EB95D02E1B96B02D009
:10631000010EB96F030EA96EB9514FEC02F019EFDF
:1063200028F0010EB95D02E1B96B02D0010EB96F20
:10633000040EA96EB9514FEC02F019EF28F0558602
:1063400055A643D055969AEC23F0030EFC5D010E42
:10635000D8A4000E316E040EFC5D010ED8A4000E10
:10636000311219E0430E92EC00F0BA0E92EC00F0FC
:10637000B80E92EC00F0BD0E92EC00F0790E92ECAB
:1063800000F0BF0E92EC00F0B80E92EC00F03E0E62
:1063900092EC00F018D0430E92EC00F0BA0E92ECA2
:1063A00000F0B80E92EC00F0BD0E92EC00F0790E09
:1063B00092EC00F0BF0E92EC00F0B80E92EC00F000
:1063C0003F0E92EC00F0E8EC3AF0BCEC39F0810EB4
:1063D000056E800E0C6E256A2368246A010E266EF7
:1063E000565028EC02F0566ED8B0E0EF25F0030EC0
:1063F000FC5D10E1810E056E400E0C6E256A23686F
:10640000246A010E266E575028EC02F0576ED8B061
:106410004FEF1FF0040EFC5D10E1810E056E400E83
:106420000C6E256A2368246A010E266E575028ECEC
:1064300002F0576ED8B03FEF1FF0810E056E200EB0
:106440000C6E256A2368246A010E266E585028ECCB
:1064500002F0586E11E2810E056E100E0C6E256A68
:106460002368246A010E266E595028EC02F0596EFA
:10647000D8B0E0EF25F064D7558655A2F4D00DECE6
:1064800017F0010EFC5D0EE1320EA96ED5514FECF6
:1064900002F0D6514FEC02F0D7514FEC02F0D85138
:1064A0004FEC02F0020EFC5D10E14EEC21F0360ED6
:1064B000A96E000E4FEC02F0000E4FEC02F0000E41
:1064C0004FEC02F0000E4FEC02F0030EFC5D1EE1FB
:1064D0004EEC21F03E0EA96E000E4FEC02F0000EC5
:1064E0004FEC02F0000E4FEC02F0000E4FEC02F009
:1064F000610EA96ED5514FEC02F0D6514FEC02F06F
:10650000D7514FEC02F0D8514FEC02F0040EFC5D75
:106510001EE14EEC21F03A0EA96ED5514FEC02F07F
:10652000D6514FEC02F0D7514FEC02F0D8514FEC5E
:1065300002F0420EA96E000E4FEC02F0000E4FEC7E
:1065400002F0000E4FEC02F0000E4FEC02F0050ED0
:10655000FC5D0EE1550EA96ED5514FEC02F0D651FF
:106560004FEC02F0D7514FEC02F0D8514FEC02F053
:10657000060EFC5D11E1FEEC06F04A0EA96E4D50D0
:106580004FEC02F04B0EA96E4F504FEC02F04C0E48
:10659000A96E51504FEC02F0070EFC5D0EE14D0E5E
:1065A000A96ED5514FEC02F0D6514FEC02F0D75105
:1065B0004FEC02F0D8514FEC02F0080EFC5D0EE1FA
:1065C000510EA96ED5514FEC02F0D6514FEC02F0AE
:1065D000D7514FEC02F0D8514FEC02F00B0EFC5D9E
:1065E00006E1650EA96E000E4FEC02F03A6A0C0E41
:1065F000FC5D24E1660EA96E000E4FEC02F0000E69
:106600004FEC02F0000E4FEC02F0000E4FEC02F0E7
:106610006A0EA96E000E4FEC02F0000E4FEC02F075
:10662000000E4FEC02F0000E4FEC02F03E6A3D6AA5
:106630003C6A3B6A436A426A416A406A9AEC23F0C8
:10664000200E92EC00F092EC00F092EC00F04F0E75
:1066500092EC00F04B0E92EC00F0030E196EE80E77
:106660005DEC02F01AD0200E92EC00F092EC00F0FB
:1066700092EC00F04E0E92EC00F06F0E92EC00F0F7
:1066800009EC3BF0070EF76ECC0EF66E8AEC00F0CC
:10669000030E196EE80E5DEC02F0E2EF25F0D896DD
:1066A000E6A9D8860AE455B007D05580558855B27A
:1066B0006CEC11F0FDEC39F002D055B055901200A1
:1066C000FE0E92EC00F0400E92EC00F00E0E92ECFA
:1066D00000F0110E92EC00F0110E92EC00F00E0E94
:1066E00092EC00F0000E92EC00F0000E92EC00F044
:1066F000000E92EC00F0000E92EC00F0FE0E92EC18
:1067000000F0480E1C6E92EC00F0070E92EC00F0C8
:10671000050E92EC00F00D0E92EC00F0000E92ECE3
:1067200000F0170E92EC00F0150E92EC00F0170E30
:1067300092EC00F0000E92EC00F0FE0E92EC00F0F5
:10674000500E1C6E92EC00F0000E92EC00F0000E69
:1067500092EC00F0000E92EC00F0000E92EC00F0D3
:106760001C0E92EC00F0140E92EC00F01C0E92EC59
:1067700000F0000E92EC00F0FE0E92EC00F0580ECD
:106780001C6E92EC00F0080E92EC00F0040E92ECFD
:1067900000F0120E92EC00F0090E92EC00F0120ED6
:1067A00092EC00F0040E92EC00F0080E92EC00F077
:1067B000000E92EC00F0FE0E92EC00F0600E1C6EEB
:1067C00092EC00F00A0E92EC00F0000E92EC00F059
:1067D0000E0E92EC00F0040E92EC00F0040E92EC1F
:1067E00000F0040E92EC00F00E0E92EC00F0000EA1
:1067F00092EC00F0FE0E92EC00F0680E1C6E92EC33
:1068000000F0080E92EC00F0040E92EC00F0120E74
:1068100092EC00F0190E92EC00F0120E92EC00F0E7
:10682000040E92EC00F0080E92EC00F0000E92ECD8
:1068300000F0FE0E92EC00F0700E1C6E92EC00F078
:106840001F0E92EC00F01F0E92EC00F0000E92EC86
:1068500000F0000E92EC00F0000E92EC00F0000E42
:1068600092EC00F0000E92EC00F0000E92EC00F0C2
:10687000FE0E92EC00F0780E1C6E92EC00F0000E12
:1068800092EC00F0000E92EC00F0000E92EC00F0A2
:10689000070E92EC00F0000E92EC00F0000E92EC6D
:1068A00000F0000E92EC00F0000E92EC00F01200EE
:1068B00080EC23F0040EFC5D04E1C00E466E090E70
:1068C000486E050EFC5D04E1C10E466E0A0E486E70
:1068D000060EFC5D04E1C30E466E0C0E486E070EFC
:1068E000FC5D04E1C50E466E0E0E486E820E056E0E
:1068F000400E0C6E4C0E236E246A086A096A200E44
:10690000016E850E20EC01F0100E20EC01F0F10E6E
:1069100020EC01F0300E20EC01F0485020EC01F0AA
:10692000010E20EC01F0000E20EC01F0000E20EC36
:1069300001F0465020EC01F0820E056E800E0C6EC8
:106940004C0E236E246A580E086E020E096E106AF1
:10695000D880DEEC00F009E300EE5AF0105018C0C9
:10696000EBFF102A10500808F3E11200A1DF558652
:1069700055A64FD055969AEC23F06050106E1052E9
:1069800019E1420E92EC00F0A50E92EC00F04D0ED3
:1069900092EC00F04B0E92EC00F0480E92EC00F0FE
:1069A000450E92EC00F0480E92EC00F04F0E92EC87
:1069B00000F015D0A90E92EC00F0420E92EC00F01F
:1069C000490E92EC00F04D0E92EC00F04B0E92EC62
:1069D00000F0480E92EC00F02E0E92EC00F009EC64
:1069E0003BF0D90E92EC00F04F0E92EC00F06E0EE0
:1069F00092EC00F0200E92EC00F04F0E92EC00F0C2
:106A0000660E92EC00F0660E92EC00F0DA0E92EC5C
:106A100000F0BCEC39F0810E056E800E0C6E256A1C
:106A20002368246A010E266E565028EC02F0566E3A
:106A3000D8A09ED7820E056E400E0C6E4C0E236EB3
:106A4000246A086A096A200E016E850E20EC01F0A6
:106A5000100E20EC01F0F10E20EC01F0300E20ECD5
:106A600001F0485020EC01F0000E20EC01F0000E87
:106A700020EC01F0000E20EC01F0FF0E4624276E02
:106A8000286AFF0E2822275020EC01F0285020EC25
:106A900001F05586D1EF2CF080EC23F0060E462451
:106AA000496E820E056E400E0C6E4C0E236E246AEB
:106AB000086A096A200E016E850E20EC01F0100EA6
:106AC00020EC01F0F10E20EC01F0300E20EC01F092
:106AD000485020EC01F0060E20EC01F0010E20ECF5
:106AE00001F0000E20EC01F0495020EC01F024DF11
:106AF0003ED780EC23F0050E4624496E820E056ECB
:106B0000400E0C6E4C0E236E246A086A096A200E31
:106B1000016E850E20EC01F0100E20EC01F0F10E5C
:106B200020EC01F0300E20EC01F0485020EC01F098
:106B3000060E20EC01F0000E20EC01F0000E20EC1F
:106B400001F0495020EC01F0F7DE11D7FD6B8CEC21
:106B500015F09AEC23F0FD5315E1A3D8E00E92EC6A
:106B600000F0650E92EC00F0BF0E92EC00F0BD0E4E
:106B700092EC00F009EC3BF0070EF76ED40EF66EC7
:106B80008AEC00F0010EFD5D15E18BD8540E92ECFD
:106B900000F0410E92EC00F0490E92EC00F0520E23
:106BA00092EC00F009EC3BF0070EF76EDE0EF66E8D
:106BB0008AEC00F0020EFD5D15E173D8540E92ECE4
:106BC00000F0570E92EC00F0410E92EC00F0540EE3
:106BD00092EC00F009EC3BF0070EF76EE80EF66E53
:106BE0008AEC00F0030EFD5D15E15BD8E00E92EC3F
:106BF00000F0700E92EC00F06F0E92EC00F0630E5D
:106C000092EC00F009EC3BF0070EF76EF20EF66E18
:106C10008AEC00F0040EFD5D15E143D8500E92ECB5
:106C200000F0410E92EC00F0420E92EC00F0530E98
:106C300092EC00F009EC3BF0070EF76EFC0EF66EDE
:106C40008AEC00F0BCEC39F0810E056E800E0C6E03
:106C5000256A2368246A010E266E565028EC02F03D
:106C6000566ED8B0E1EF2AF0810E056E200E0C6E44
:106C7000256A2368246A010E266E585028EC02F01B
:106C8000586E21E2810E056E100E0C6E256A236887
:106C9000246A010E266E595028EC02F0596E0EE25D
:106CA00056D7E00E92EC00F0610E92EC00F0BF0EB1
:106CB00092EC00F02E0E92EC00F01200040EFD5D3E
:106CC000D8A0FD2B44D7FD53D8A4FD0740D75F5073
:106CD000BC6F6050BB6F35D0080E49EC02F0106EEF
:106CE000105205E16D50BC6F6E50BB6F04D0615007
:106CF000BC6F6250BB6F25D0080E49EC02F0106EDD
:106D0000105205E17150BC6F7250BB6F04D06F50D0
:106D1000BC6F7050BB6F15D0080E49EC02F0106EBE
:106D2000105205E16750BC6F6850BB6F04D06B50C8
:106D3000BC6F6C50BB6F05D06950BC6F6A50BB6FA5
:106D400000D0BBC014F0BCC015F0166A176A1F6AE9
:106D5000070E1E6EA10E1D6E200E1C6EFAEC02F0C8
:106D600017C02AF016C029F015C028F014C027F06B
:106D70002AC017F029C016F028C015F027C014F05B
:106D80001F6A1E6A040E1D6E1C6A74EC02F017C0A6
:106D9000DCF016C0DBF015C0DAF014C0D9F0DCC0AE
:106DA00017F0DBC016F0DAC015F0D9C014F01F6A76
:106DB000010E1E6E860E1D6EA00E1C6E74EC02F08F
:106DC00014C0C1F0DCC017F0DBC016F0DAC015F05B
:106DD000D9C014F01F6A010E1E6E860E1D6EA00E25
:106DE0001C6E74EC02F01FC0DCF01EC0DBF01DC096
:106DF000DAF01CC0D9F0800E016EC15132EC00F007
:106E00002C0E92EC00F0050E0B6EDCC02AF0DBC0FD
:106E100029F0DAC028F0D9C027F063EC00F0420E68
:106E200092EC00F01200FD6BF66B050EF76F9AEC1A
:106E300023F0FD5343E18DEC23F0A40E92EC00F01F
:106E4000B30E92EC00F0E30E92EC00F0480E92ECE0
:106E500000F06F0E92EC00F0BC0E92EC00F0650EAC
:106E600092EC00F0700E92EC00F0440E92EC00F008
:106E7000450E92EC00F04D0E92EC00F04F0E92ECAD
:106E800000F0820E056E400E0C6E4C0E236E246ACE
:106E9000086A096A200E016E820E20EC01F0100EC5
:106EA00020EC01F0F10E20EC01F01A0E20EC01F0C4
:106EB000910E20EC01F02E0E20EC01F0010EFD5D94
:106EC00040E18DEC23F04B0E92EC00F06F0E92EC53
:106ED00000F0E30E92EC00F0200E92EC00F0450E74
:106EE00092EC00F0A00E92EC00F04B0E92EC00F051
:106EF000440E92EC00F0450E92EC00F04D0E92EC38
:106F000000F04F0E92EC00F0820E056E400E0C6EFB
:106F10004C0E236E246A086A096A200E016E820EE6
:106F200020EC01F0100E20EC01F0F10E20EC01F04D
:106F30001A0E20EC01F0920E20EC01F02F0E20EC46
:106F400001F0020EFD5D43E18DEC23F0A80E92EC02
:106F500000F0700E92EC00F06F0E92EC00F0C10E9B
:106F600092EC00F0B80E92EC00F0B30E92EC00F050
:106F7000BA0E92EC00F0610E92EC00F0440E92EC2E
:106F800000F0450E92EC00F04D0E92EC00F04F0E2A
:106F900092EC00F0820E056E400E0C6E4C0E236ECD
:106FA000246A086A096A200E016E820E20EC01F044
:106FB000100E20EC01F0F10E20EC01F01A0E20EC86
:106FC00001F0940E20EC01F0310E20EC01F0820E65
:106FD000056E800E0C6E4C0E236E246A2C0E086E0D
:106FE000010E096E106AD880DEEC00F009E300EEB5
:106FF0008AF0105018C0EBFF102A10502F08F3E150
:107000008A51F36FF39DF39F020EF327F653D8A432
:1070100064D0070EF96F0C0EF75D1BE2F7510C08F8
:107020000F6E010EF86FF8510F5C03E3F907F82BB0
:10703000FAE1050EFA6F050EF9250F6EFAC0F8F0A9
:10704000F8510F5C05E3F851F35D02E3F82BF8E12A
:1070500037D0070EF75DFA6F070EFA250F6EFAC0EC
:10706000F8F0F8510F5C0EE3F851F35D0BE300EE1E
:107070008AF0F851EB50106E105200E1F8C0F9F0B0
:10708000F82BEFE1070EFA25276E286A2836F9510A
:10709000275C106E000E2858116E105202E111523A
:1070A0000FE0070EFA25276E286A2836F951275C6B
:1070B0000F6E010EF86FF8510F5C02E3F82BFBE145
:1070C000F72B070EF325106E116A1136115205E1E8
:1070D000F751105C02E2050EF76FF62B050EF65D18
:1070E000D8B4F66B49D9810E056E800E0C6E256AF8
:1070F0002368246A010E266E565028EC02F0566E64
:10710000D8B0E1EF2AF0810E056E200E0C6E256AD4
:107110002368246A010E266E585028EC02F0586E3F
:107120000FE2810E056E100E0C6E256A2368246A2C
:10713000010E266E595028EC02F0596E05E266D712
:10714000FD53D8A4FD0770D6020EFD5DD8A0FD2B1F
:107150006BD6E68102EC3BF0FF5303E1EDEC11F05E
:1071600071D8FF5322E06CEC11F0010EFE6F010E9E
:10717000FF5DD8B419EC18F0020EFF5DD8B4E1EC55
:107180001AF0030EFF5DD8B4A5EC1AF0040EFF5DF3
:10719000D8B433EC1AF0050EFF5DD8B497EC1DF0AF
:1071A000060EFF5DD8B490EC19F078D855B24FECCC
:1071B00033F081A604D0A7EC14F062EF06F0640E61
:1071C0005CEC02F0810E056E800E0C6E256A236861
:1071D000246A010E266E565028EC02F0566ED8B086
:1071E000A9EF13F0810E056E400E0C6E256A236820
:1071F000246A010E266E575028EC02F0576ED8B064
:10720000B5D0810E056E200E0C6E256A2368246AA7
:10721000010E266E585028EC02F0586ED8B056EF8A
:1072200015F0810E056E100E0C6E256A2368246A17
:10723000010E266E595028EC02F0596ED8B06CEF52
:1072400015F088D738C014F039C015F00A0E186E42
:10725000196AE3EC02F0C56F15C0C6F0C5C014F0A2
:10726000C6C015F0E80E186E030E196EE3EC02F0BE
:10727000C16FC5C014F0C6C015F0E80E186E030E3D
:10728000196EE3EC02F01CC0C5F01DC0C6F0080E7C
:10729000F76E060EF66E8AEC00F01200BAD90A0EEE
:1072A000FC5D35E1C7C014F0C8C015F00A0E186EB9
:1072B000196AE3EC02F0C16FC7C014F0C8C015F042
:1072C0000A0E186E196AE3EC02F01CC0C2F0DA0E66
:1072D00092EC00F02D0E92EC00F00A0EC15D03E27C
:1072E000200E92EC00F0800E016EC15132EC00F0E5
:1072F0002C0E92EC00F0010E0B6EC25133EC00F03C
:107300002B0E92EC00F0D90E92EC00F02ED0DA0E9B
:1073100092EC00F02D0E92EC00F0030EC85DE80E2A
:10732000D8B4C75D03E2200E92EC00F0C85306E12A
:10733000640EC75D03E2200E92EC00F0C85306E134
:107340000A0EC75D03E2200E92EC00F0800E016E83
:107350000B6AC7C01CF0C8C01DF035EC00F02B0E46
:1073600092EC00F0D90E92EC00F01200FF2B070E09
:10737000FF5DD8B4FF6BEED655B24FEC33F081B65B
:1073800062EF06F0640E5CEC02F012009AEC23F05F
:1073900027D83FD9A90E92EC00F0BA0E92EC00F07B
:1073A000700E92EC00F0610E92EC00F0040E92EC84
:1073B00000F0BD0E92EC00F0610E92EC00F0030EB6
:1073C000196EE80E5DEC02F0080EF76E100EF66E08
:1073D0008AEC00F0070E196ED00E5DEC02F0120080
:1073E000A00E92EC00F04B0E92EC00F0080EF76E3F
:1073F0001A0EF66E8AEC00F0120055A4E8D0755013
:10740000106E10C0BEF0BD6B7650106E1050BD13E4
:107410006F50106E10C0C0F0BF6B7050106E1050E7
:10742000BF13020E49EC02F0C16F030E49EC02F0EB
:10743000C26F010EC25D02E0020EC26FD890BD3570
:10744000276EBE35286E296A29362A6A2AC017F0A7
:1074500029C016F028C015F027C014F01F6A1E6A54
:107460001D6AC2C01CF0FAEC02F017C0D2F016C0C0
:10747000D1F015C0D0F014C0CFF0D2C017F0D1C0F9
:1074800016F0D0C015F0CFC014F0BFC01CF0C0C0C3
:107490001DF01E6A1F6AFAEC02F017C0D2F016C087
:1074A000D1F015C0D0F014C0CFF0D2C017F0D1C0C9
:1074B00016F0D0C015F0CFC014F01F6A1E6A1D6A06
:1074C000C1C01CF0FAEC02F017C0D2F016C0D1F027
:1074D00015C0D0F014C0CFF0D2C017F0D1C016F054
:1074E000D0C015F0CFC014F01F6A050E1E6E7E0EC0
:1074F0001D6E400E1C6E74EC02F017C0D2F016C068
:10750000D1F015C0D0F014C0CFF0CF51CD27D0515D
:10751000CE23030ECE5D23E303E1E80ECD5D1FE332
:10752000CDC014F0CEC015F0E80E186E030E196E23
:10753000E3EC02F0276E15C028F02750D32728501F
:10754000D423CDC014F0CEC015F0E80E186E030E93
:10755000196EE3EC02F01CC0CDF01DC0CEF08151DD
:10756000106E10503A5C02E281513A6E8151106EF9
:10757000060E105C2CE38151106E10503B243B6EC4
:10758000000E3C203C6E000E3D203D6E000E3E2065
:107590003E6E402A000E4122422243223EBE17D0B8
:1075A000770E3E5C14E30BE1350E3D5C10E307E122
:1075B000940E3C5C0CE303E1000E3B5C08E33E6A86
:1075C0003D6A3C6A3B6A436A426A416A406A120009
:1075D00020D8D90E92EC00F0540E92EC00F0610E1F
:1075E00092EC00F0BA0E92EC00F0200E92EC00F05B
:1075F000480E92EC00F0690E92EC00F0DA0E92EC7C
:1076000000F01200FE0E92EC00F0020E92EC00F080
:107610001200FE0E92EC00F0C00E92EC00F0120090
:02762000FFD792
:020000040030CA
:0E000000FFF2E2EEFFFDBBFFFFFFFFFFFFFF81
:00000001FF
